:020000040800F2
:10500000A01C0020D55000085192000845880008D7
:105010000000000000000000000000000000000090
:1050200000000000000000000000000049A500088A
:105030000000000000000000899B0008E5A60008B1
:10504000E7500008E7500008E7500008E750000864
:10505000E7500008415C0008E7500008E7500008EE
:1050600000000000E7500008315B0008E75000082E
:10507000E7500008698D000800000000E7500008B4
:1050800000000000E75000080000000000000000E1
:10509000E750000800000000E7500008E750000853
:1050A000E7500008E7500008E7500008E1B20008A8
:1050B000E7500008E7500008000000000000000072
:1050C0000348854600F07EFC0048004705C4000800
:1050D000A01C00200448804704480047FEE7FEE784
:1050E000FEE7FEE7FEE7FEE7A5A70008C1500008BF
:1050F00030B50B46014600202022012409E00D4670
:10510000D5409D4205D31D469540491B25469540F7
:1051100040191546521E002DF1DC30BD70B500243B
:105120002546002801DA01244042002901DA012540
:105130004942FFF7DDFFAC4200D04042002C00D0D6
:10514000494270BDF0B51FB40646002082B0054646
:105150004024019100901BE0019922460F46304601
:1051600000F06CFB049A059B801A994110D31046FD
:105170001946224600F052FB361A8F41019722460B
:1051800001200021009F00F049FB38184D4100909C
:105190002046641E0028DFDC019B00982946324629
:1051A00007B0F0BD03460B439B0703D009E008C9D5
:1051B000121F08C0042AFAD203E00B780370401CC7
:1051C000491C521EF9D27047D2B201E00270401C55
:1051D000491EFBD270470022F6E710B513460A4677
:1051E00004461946FFF7F0FF204610BD30B50446CF
:1051F0000020034600E05B1C934203D2E05CCD5CE0
:10520000401BF8D030BDF8B502464A40D40F4200EA
:105210004B0052085B089A4202D2024608461146E9
:105220004A0023D0C30D4A00DDB2120EAD1A202D64
:1052300035DA49020126490AF6058A19002C00D000
:10524000524220214F1B1146B9402A411018C20D6D
:105250009A4221D0002C17D0012D08DCDA05801AE3
:10526000D20F8019D207DBB200F014FBF8BDDA05CB
:10527000801A012340001B06C01880185A4280186B
:10528000CA0F1043490007E04908C2071143DA0575
:10529000801A80194008801800F0F4FAF8BD610007
:1052A0000122511A001BF7E70122D2075140AAE759
:1052B0000122D2075040A6E770B502464A40D50FFA
:1052C00040004A00ED0740085208002814D0002A88
:1052D00012D0C40DD30D41020120C0055202490A6B
:1052E000520AE41A091812187D34914201D3641C41
:1052F00000E04900002C01DA002070BD002391423B
:1053000001D3891A0343400849000028F7D1002936
:105310000AD0914202D10121C90705E0914201D290
:10532000012101E00121C943E005C018401900F046
:10533000A9FA70BDF0B507460846584087B0C00FBF
:10534000049048000E46590040084908BC1A88419C
:1053500005D2384631461E4617460B4602465800CF
:10536000400810434CD0300D039040055900400DCB
:10537000490D0590401A0290402872DA1803012165
:10538000000B09050843019004980092002805D0FD
:1053900001995242002088410092019002984021D8
:1053A0000A1A0199009800F039FA05460C466B4636
:1053B00007CB00F054FAC0197141039A0E0D002377
:1053C000D71756401A467A40164344D0049A002A0A
:1053D0002DD0029A012A039A15DC1205C01A9141B8
:1053E00001263605001C7141D20F059ED20700939D
:1053F000019202962A46234600F092FA07B0F0BDC9
:1054000038463146FAE71605224A0F46B218C01A46
:10541000B74101210905001C4F4100187F41114689
:1054200018187941E20F10436D19644113E0E20747
:105430006D0815436408C2071443039A0126120538
:10544000C01A91413605001C7141CE074008304317
:105450004908C01851412A46234600F054FACDE7C6
:10546000FFE7049801224000C117121A00238B4164
:1054700004983146C417381AA141EEE730B401242C
:10548000E407634030BC55E730B40124E4076140D1
:1054900030BC4FE70000E0FFF0B51FB488B00B99B7
:1054A0000998002448400999C00F4900490809910A
:1054B000C0070B990090490049080B910999089879
:1054C000A64608431CD00B990A98084318D009989F
:1054D00001244000420D4800410D099824050003B5
:1054E000000B204309900B980003000B20430B9006
:1054F00050181C494018002201901446104605E03F
:10550000002001460DB0F0BD032801DA034600E09B
:1055100003239C46C11A0AAE0AE05F0008ADED5BAA
:105520004F00F75B7D430027AA187C41491C5B1E96
:105530006145F2DD410004AB5A522104120C0A43CA
:10554000240C401C0828DFDB01980290009970466B
:1055500001910090059B049A0799069800F0E0F9E4
:10556000D0E700000DFCFFFFF0B50C465C4085B0B5
:10557000E40FE40703944C000026640859009446A5
:10558000490802460296224321D062460A431ED0B1
:105590006200570D4A000E032303550D01240246F5
:1055A0002C492405781B1B0B360B4018234326433C
:1055B000614600901C46501AB44103D30098401C29
:1055C000009002E0921800985B41002803DA002066
:1055D000014605B0F0BD00200121090507468646B9
:1055E00011E064461D46141BB54106D36546521BA7
:1055F000B341744607430C43A646CD07400849080B
:10560000284392185B4105460D43EAD110461843E2
:1056100013D06046194650407140084306D060469A
:10562000101AB34106D20122002306E00022012312
:10563000DB0702E00122D2435310009874460105B3
:10564000381C6141029C039D0019694100F05BF91F
:10565000BFE70000FD030000C217C10F504010B5A6
:105660004018CA079623002100F014F910BD10B5A8
:1056700000229623114600F00DF910BD0EB5C21799
:10568000C10F5040CA0740180021054B02930192F8
:1056900000910A460B4600F043F903B000BD00003C
:1056A000330400000EB505490291002100910A461D
:1056B0000B46019100F034F903B000BD3304000043
:1056C000410040020122400AD205090E80187F29BC
:1056D00001DA00207047962903DC9622511AC8404F
:1056E000704796398840704770B5CD0F4A0009035E
:1056F0000123090B1B0519430B4BED070024520D29
:105700009A4201DA002070BD074B34339A4203DC21
:105710009A1A00F093F802E00449511888402C438B
:10572000F1D0404270BD0000FF030000CDFBFFFF41
:105730004A0009030123090B1B051943094B10B546
:10574000520D9A4201DA002010BD064B34339A42C2
:1057500003DC9A1A00F072F810BD03495118884012
:1057600010BD0000FF030000CDFBFFFFC20FD207FA
:10577000400040080BD0C10D0723DB01C9184002CF
:105780000905400A1143C208400711437047002031
:105790000146704710B5002904DB0124E4074042AC
:1057A0008C412146002B04DB1C460123DB075242BF
:1057B000A341994200D1904210BD0000CB0FDB07FE
:1057C000490010B5490802460A4307D00A0D0724CC
:1057D0000903E401090B121B002A01DC002010BDA3
:1057E000C900440F0C43C100E018D205801800F036
:1057F00049F810BD0122D207002800DB101A002949
:1058000000DB511A814270470122D207002800DBD9
:10581000101A002900DB511A8842704710B5202A5F
:1058200004DB0146203A9140002010BD9140202326
:105830009C1A0346E3401943904010BD10B5202A3E
:1058400004DB0846203AD040002110BD0B46D3406F
:10585000D0402024A21A91400843194610BD10B52B
:10586000202A06DBCB170846203A1041C1170B430C
:1058700006E00B461341D0402024A21A9140084371
:10588000194610BD002904DA401C490001D1400826
:105890004000704770B40024050C05D110240004AA
:1058A00002D1002921D01124050E01D100020834B3
:1058B000050F01D10001241D850F01D18000A41C1A
:1058C000002801DB4000641C002908D020252E1B85
:1058D0000D46F540A14000D00121294308430106AF
:1058E0001B1B000ADB1D02D5002070BC7047DB05C6
:1058F000181880180029F8DA401C4900F5D170BC4E
:1059000040084000704710B5002B08DA0024401C06
:10591000614192185B411A4301D14008400010BD1B
:10592000F0B51FB482B005460C0003D0084605F060
:1059300003FE02E005F000FE203002460090214602
:105940002846FFF76BFF049B059A04460F46184351
:105950001143084314D0184610431BD0009840212F
:105960000A1A18460599FFF769FF05460E46009A80
:1059700005990498FFF752FF084305D0012004E081
:105980002046394607B0F0BD0020C11705430E433D
:105990002C43374300990E986305401A7905E40AB1
:1059A00000220C43FD0A0A3002D500200146E9E737
:1059B0000105101969410C9C0D9D00196941FFF703
:1059C000A2FFDFE7064C0125064E05E0E36807CCA1
:1059D0002B430C3C98471034B442F7D3FFF774FBC9
:1059E000ECC700080CC8000870B58C180578401C7E
:1059F0006B075B0F01D10378401C2A1106D1027896
:105A0000401C03E006780E70401C491C5B1EF9D157
:105A10002B0705D40023521E0DD40B70491CFAE746
:105A20000378401CCB1A921C03E01D780D70491CB2
:105A30005B1C521EF9D5A142D8D3002070BD0000D6
:105A400038B50446074908480068FFF751FB604332
:105A5000009002E00098401E009000980028F9D1C4
:105A600038BD000040420F00B801002070B5044668
:105A70000025206880688007800F012807D12068F2
:105A80000068C007C00F002801D0012000E00020FE
:105A9000002839D1206880681C490840002801D1BD
:105AA000012000E00020002809D1606D102108438A
:105AB0006065A06D01210843A065012070BD2068CC
:105AC000806801210843216888600120FFF7B8FF42
:105AD00001F0E0F905460EE001F0DCF9401B0A2870
:105AE00009D9606D102108436065A06D012108434C
:105AF000A0650120E2E720680068C007C00F01210F
:105B0000484048400028E7D00020D7E71700008031
:105B100010B502460B460020002103E0545C241817
:105B2000A0B2491C9942F9D3C443A0B210BD0000F1
:105B300010B5034800F0A8FE024800F0A5FE10BD15
:105B40003C180020F417002030B51C25446C2C4074
:105B50000125A540046C6560046863608468102CAE
:105B600004D10468A2600468E16003E00468A160F5
:105B70000468E26030BD000001201D494872022027
:105B80001C49487203201C49487204201B49487272
:105B900017481B490978017017481949097801709D
:105BA0001448174909780170114816490A7842715A
:105BB00049788171104813490A7842714978817196
:105BC0000C4810490A784270497881700B480D4999
:105BD0000A784270497881700B480A490A78427005
:105BE0004978817007490A78427149788171704714
:105BF000EC1100204A1200200E120020001200209A
:105C000063010020580100206012002010B504F04C
:105C10006FFC202004F054FD012006F0A9F80020BC
:105C200004F04EFD044805F011FF044806F056FA52
:105C3000002006F093FA10BD690000208380000068
:105C400010B501210520000701F010F9002802D04D
:105C50000020174908600221164801F007F90028C2
:105C60001FD10120144908701448808F00280DD0DE
:105C70000022012189020F4801F005F90A2005F0F0
:105C800093FE012291020B4801F0FDF80020084923
:105C900008600B4800880A2148430A49088005F03B
:105CA00031FB012000F0DCFF022000F0D9FF10BD25
:105CB000A801002000040050B0010020EC0D0020DD
:105CC000740100209C0100207047000000210A4A56
:105CD00051610A494968012252021143074A516041
:105CE0001146496808221143044A51600021C20943
:105CF000D20111607047000084180020002002408B
:105D00007FB504460D460020039000F061FF00209F
:105D100000900194E809029003A9684600F0DAFEB9
:105D2000002804D000F01CFF002004B070BD00F07B
:105D300017FF0120F9E710B50346002002E01C5CC4
:105D40000C54401C9042FAD310BD00000020394989
:105D50008969FF2201321140914208D136494969CF
:105D600002221143344A5161FF2101310843314974
:105D70008969012252021140914208D12E49496994
:105D8000012211432C4A516101214902084329494A
:105D90008969012292021140914208D1264949693C
:105DA00008221143244A51610121890208432149F3
:105DB00089690122D2021140914208D11E494969E4
:105DC000042211431C4A51610121C90208431949A7
:105DD0008969012252031140914208D1164949694B
:105DE00010221143144A516101214903084311490A
:105DF0008969012252041140914207D10E49496933
:105E0000202211430C4A5161202108430949896924
:105E1000012212041140914208D1074949694022E8
:105E20001143054A51610121090408430149886170
:105E300070470000002002408418002070B504461E
:105E400001F028F805460BE0601C002808D0002C63
:105E500004D001F01FF8401BA04201D9032070BDFF
:105E60001F488069C007C00F0028EDD11C48806919
:105E700002210840022801D1194988611848806927
:105E8000FF2101310840884223D01548806949002C
:105E9000084088421DD01248806949000840884265
:105EA00017D00F48806949000840884211D00C483B
:105EB00080698900084088420BD00948806909013F
:105EC0000840884205D00648806949100840884249
:105ED00003D1FFF73BFF0120C1E70020BFE700002F
:105EE00000200240F0B585B006460F461446002556
:105EF000029601970020009000F06AFE13E00198DE
:105F0000006803900220039A029900F039FE009085
:105F10000098002800D008E00298001D0290019827
:105F2000001D01902D1DA542E9D300BF00F018FE11
:105F3000A54202D2002005B0F0BD0120FBE7000021
:105F40000246002108E04800064B185A904201D151
:105F500008467047481CC1B2034800788142F2DB12
:105F600000BFF6E75A1400203001002070B5044647
:105F70000D462946204600F082FF70BDFEB50C4854
:105F800001F024FA80B202900298FFF78BFB0446DE
:105F9000084A094BFFF780FA0022084B0191009054
:105FA000FFF7E2FA0646FFF7C3FB80B2FEBD000032
:105FB000EC160020F853E3A59B843E4000408F4040
:105FC00010B5364836490A784270497881703549AB
:105FD0000A784271497881710520304948720A2057
:105FE00006F06AF87D20C00006F082F800222B49F6
:105FF0000C2006F07FF900210C2006F08FF902201A
:1060000006F0B4F800BF00210F2005F0B3FF2649C9
:106010000860264908400028F5D023480068401C45
:10602000002801D103F052F91F48006801218903BB
:106030000840002831D08122D20100210F2006F033
:1060400012F90021102005F095FF4406640E214648
:106050000022174805F0DEFF1548407A05281CD1BC
:10606000022210491248401DFFF7C0F8002814D141
:106070000F48807C0F49087004220D49491C0E48C6
:10608000FFF790F80B4800784200094913310B489C
:10609000FFF788F803200A49087010BD601200203D
:1060A0000A010020580100207800002000D0272499
:1060B000B012002030010020380100205A140020C6
:1060C0006800002010B50B4800F074FB0A21094855
:1060D00000F0FAFA074800F0A1F90121490208404E
:1060E000884204D1034800F09CF980B210BD00BF83
:1060F000FCE7000090160020F0B587B000220121D7
:10610000424800F0C0FEFFF7DDFF0546FFF7AFFA9B
:1061100004463F49FFF7D0F83E4908600122114686
:106120003A4800F0B0FE3B480068FFF71FFB04460A
:106130000022394BFFF72EFB5ED838480078002844
:1061400021D0002035490870FFF7BCFF0546FFF756
:106150008EFA04462E49FFF7AFF82E49086008462C
:106160000068FFF703FB044600222B4BFFF786F97C
:1061700000222B4B05910490FFF78EF90646FFF79E
:106180001DFB2849086023480068FFF7EFFA064620
:106190000022214BFFF772F90446234A234BFFF7F5
:1061A0007BF9039102901F480068FFF7DFFA04466D
:1061B0001D4A52421E4BFFF76FF901910090039B5D
:1061C000029AFFF7B7F805910490FFF7F7FA15491F
:1061D0000860184913480068FFF716FB02D21548FB
:1061E0001049086000210F480068FFF703FB06D242
:1061F00000200C49086002E000200A4908600948B4
:106200000068FFF75DFAC0B207B0F0BD00040050AF
:1062100000401B443000002000000C4038000020EB
:1062200000E06440340000203333333333B3304074
:10623000CCCCEC3F0000C842F8B50446002500264F
:10624000002700BF5020005D012801D10220F8BDC9
:1062500001215020015500BF206880688007800F11
:10626000012806D1206800680840002801D00120DC
:1062700000E00020002841D1606DFF2101318843FA
:106280000221084360652068C0688707BF0F206847
:10629000C068800880002168C8602068806801218B
:1062A000C90708432168886000F0F4FD064611E044
:1062B00000F0F0FD801B0A280CD9606D0221884394
:1062C00010210843606500BF00215020015500BF28
:1062D0000120BCE720688068C00FC0070121C90702
:1062E0008842E5D02068C06838432168C860606D86
:1062F0000221884301210843606504E0606D20218C
:1063000008436065012500BF00215020015500BFF2
:1063100028469CE770B504460D4600BF5020005D3E
:10632000012801D1022070BD01215020015500BF7C
:106330002068806804210840800800280AD0606D29
:1063400020210843606500BF00215020015500BF97
:106350000120E8E72D496868884229D02068806AD2
:1063600029684903490B084321688862286840036B
:10637000400B2749084001218904884208D125485B
:10638000806849010843234988600A20FFF758FBC9
:1063900028684003400B20490840012149048842F5
:1063A0002CD11C488068490108431A49886025E0BF
:1063B0002068806A29684903490B884321688862FC
:1063C00028684003400B1249084001218904884293
:1063D00005D110488068490188430E4988602868C3
:1063E0004003400B0C49084001214904884205D173
:1063F00008488068490188430649886000BF002139
:106400005020015500BF00208DE700000110000062
:106410000000044800270140000002440146486D86
:10642000704701460868006C7047000010B50446CC
:10643000002C01D1012010BD606D002806D1A0659F
:10644000002150200155204600F00EF9606D10210A
:106450000840102806D02068806804210840800881
:1064600000280AD0606D10210843606500BF00213C
:106470005020015500BF0120DDE7606DFF21013193
:106480008843022108436065206880688007800F88
:10649000012807D120680068C007C00F002801D07C
:1064A000012000E0002000283AD100BF0321890725
:1064B0006068884207D049426068884203D049003A
:1064C000606888420CD120680069800080082168DB
:1064D000086120680069616808432168086112E06A
:1064E0002068006980008008216808615C48806835
:1064F0000F21890488435A4988600846806861688A
:1065000008435749886000BF2068C0681821884345
:106510002168C8602068C068A16808432168C86015
:106520004F4880680121490688434D4988600846E4
:106530008068A18E490608434949886020688068C0
:10654000012109070840002804D120688068084319
:10655000216888602068C068424908402168C86096
:106560002169E068022901D1042100E000210843EB
:106570002021095D490308432C21095D4900084396
:10658000216B0843A16989030843E169C9030843F2
:106590002168C96808432168C860FF21C231606A68
:1065A000884207D0A16A606A08432168C968084325
:1065B0002168C8602120005D012813D12020005DE2
:1065C000002807D12068C068012109040843216818
:1065D000C86007E0606D202108436065A06D01215F
:1065E0000843A065E06B012817D120680069FF21EE
:1065F0008900884321680861216C606C0843A16CA4
:106600000843216809690843216808612068006916
:1066100001210843216808610BE020680069C00778
:10662000C00F002805D0206800694008400021689C
:10663000086120684069C008C0002168486120687E
:106640004069A16B0843216848610020A065606D26
:10665000022188430121084360650020EBE6000029
:10666000002701401902FEFF10B586B00446142130
:1066700001A8FEF7B0FD1249206888421ED11148DA
:10668000406B491508430F49486300BF0846C06A7C
:10669000012108430B49C8620846C06AC007C00F01
:1066A000009000BF00BF0220019003200290002054
:1066B000039001A90520000700F0E2FA06B010BD22
:1066C0000024014000100240F8B504460D460026A3
:1066D00000276069082801D1082711E02068C068F8
:1066E000C007C00F00280AD0606D202108436065F4
:1066F00000BF00215020015500BF0120F8BD0C272C
:1067000000F0C8FB064614E0681C002811D0002DDC
:1067100004D000F0BFFB801BA8420AD9606D0421A1
:106720000843606500BF00215020015500BF0320D1
:10673000E4E72068006838400028E5D0606D01215A
:106740004902084360652068C06803218902084047
:10675000002826D12020005D002822D12068006872
:106760000821084008281CD12068806804210840BE
:10677000800800280DD1206840680C2188432168DA
:106780004860606DFF210131884301210843606545
:1067900007E0606D202108436065A06D012108437A
:1067A000A065A069002802D10C20216808600020A3
:1067B000A4E7000070B50446002520688068042125
:1067C0000840800800282BD100BF5020005D012820
:1067D00001D1022070BD01215020015500BFE069A8
:1067E000012803D02046FFF741F90546002D18D1B6
:1067F000606D0D490840FF210131084360650020AC
:10680000A06500BF00215020015500BF1C20216859
:10681000086020688068042108432168886000E0DF
:1068200002252846D6E70000FEF1FFFF70B50446BA
:1068300000252520005D022803D00420E063012507
:1068400020E0206800680E218843216808602068E5
:10685000006840084000216808601C21606C084006
:1068600001218140206C416001212520015500BF9C
:1068700000212420015500BFA06B002802D0204633
:10688000A16B8847284670BD70B50446206C05682A
:10689000206806681C20616C014004208840284064
:1068A00000281DD004203040002819D0206800683E
:1068B00020210840002805D1206800680421884371
:1068C000216808601C21606C084004218140206C14
:1068D0004160206B00285AD02046216B884756E043
:1068E0001C20616C0140022088402840002825D0EF
:1068F00002203040002821D0206800682021084074
:10690000002808D1206800680A21884321680860AF
:106910000121252001551C21606C08400221814085
:10692000206C416000BF00212420015500BFE06AB7
:1069300000282CD02046E16A884728E01C20616CA2
:106940000140082088402840002820D008203040FE
:1069500000281CD0206800680E2188432168086048
:106960001C21606C084001218140206C41600120A5
:10697000E06301212520015500BF0021242001559D
:1069800000BF606B002802D02046616B884770BD55
:1069900070B50446002C01D1012070BD244A216845
:1069A000881A1421FEF7A4FB800060642048083890
:1069B0002064022125200155206805681D480540F6
:1069C000E168A06808432169084361690843A16937
:1069D0000843E1690843216A0843054320680560CC
:1069E00001218903A068884217D011487830806A55
:1069F0001C22616C11400F228A4090430C4978316F
:106A000088621C22616C11406068884008497831B6
:106A1000896A08430649783188620020E0630121D1
:106A2000252001550021242001550020B5E7000054
:106A3000080002400F80FFFFF8B504460D461646D9
:106A40001F460020009000BF2420005D012801D1D6
:106A50000220F8BD01212420015500BF2520005D42
:106A600001282DD10221252001550020E063206856
:106A7000006840084000216808603B4632462946CD
:106A80002046FFF761F8206B002806D020680068D8
:106A90000E210843216808600BE02068006804218B
:106AA000884321680860206800680A21084321683B
:106AB000086020680068012108432168086006E03A
:106AC00000BF00212420015500BF02200090009843
:106AD000BFE70000F8B504460E460127002500BFB9
:106AE0001C48007C012801D10220F8BD0120194971
:106AF000087400BF1848FFF7A1F90746002F22D1FC
:106B0000401E3060656817E02846FFF7DFF812483E
:106B1000FFF794F9074611484068082188430F4958
:106B2000486008464068491588430C494860002F72
:106B300001D0356006E08035A068C001616840186A
:106B4000A842E1D800BF00BF00200249087400BF7E
:106B50003846CAE78418002050C3000000200240D5
:106B600006484068022108430449486008464068D6
:106B7000012108430149486000207047002002407D
:106B8000F8B507460C461546012600BF0E48007CA6
:106B9000012801D10220F8BD01200B49087400BF73
:106BA0000A48FFF74BF90646002E06D10649486110
:106BB00025600648FFF742F9064600BF002002495B
:106BC000087400BF3046E6E78418002050C3000078
:106BD0001D484068C007C00F002816D000BFEFF363
:106BE0001080014600BF72B61848174AD060184896
:106BF000D06000BF81F3108800BF10464068C00716
:106C0000C00F002801D0012070470F4840680222C1
:106C10001040022815D100BFEFF31080014672B674
:106C20000C48094A10610C481061084680F310882E
:106C300000BF1046406802221040022801D1012006
:106C4000E2E70020E0E7000000200240EFCDAB8942
:106C500005040302BFAE9D8C161514137047000087
:106C600010B50446054840692040002804D0034878
:106C700044612046FFF7F2FF10BD00000004014010
:106C800070B50346002200240020DAE00126964079
:106C90000D6835402C46002C77D04D68022D02D06F
:106CA0004D68122D15D1D508AE001D462035A859C6
:106CB0005507EE0E0F25B5400646AE433046560743
:106CC000F60E0D69B5402843D508AD001E462036A6
:106CD00070514D68012D08D04D68022D05D04D68CA
:106CE000112D02D04D68122D18D198685600032539
:106CF000B5400646AE4330465600CD68B540284301
:106D000098605868012595400646AE4330461026E7
:106D10004D6835402D099540284358601868560045
:106D20000325B5400646AE4330460D79AD07AD0F9D
:106D30005600B54028431860D86856000325B54072
:106D40000646AE43304656008D68B5402843D860AD
:106D5000012636074D683540B54271D13C4D6D6B0B
:106D6000012635433A4E75633A4D9608B600A85948
:106D700095072E0F0F25B5400646AE433046052534
:106D80002D07AB4202D1002515E059E0324DAB4250
:106D900001D101250FE0314DAB4201D102250AE0BE
:106DA0002F4DAB4201D1032505E02E4DAB4201D161
:106DB000052500E006259607360FB5402843254DEA
:106DC0009608B600A851284D28680546A5432846D0
:106DD000012636044D683540B54202D105462543AB
:106DE0002846214D286068680546A54328460126A7
:106DF00076044D683540B54202D105462543284604
:106E0000194D6860A8680546A54328460126360541
:106E10004D683540B54202D1054625432846124DFE
:106E2000A860E8680546A5432846012676054D6812
:106E30003540B54202D10546254328460A4DE86053
:106E4000521C0D68D540002D00D01FE770BD00001A
:106E500000100240080001400004005000080050EB
:106E6000000C0050001C0050000401400246136951
:106E70000B40002B01D0012000E000207047426948
:106E80004A4042617047002A01D0816100E081627E
:106E9000704700000148006870470000B4010020FE
:106EA00002480068401C014908607047B401002096
:106EB00010B50024084800684021084306490860CE
:106EC000002000F00BF8002801D0012401E000F0C0
:106ED000B3FA204610BD00000020024070B5044601
:106EE00000257D21C90009480068FEF701F9064622
:106EF00001F062F9002801D0012504E000222146BA
:106F0000501E00F0C1FA284670BD0000B8010020F4
:106F10007047704770B506467E480078401C7D4932
:106F2000087001207C4908707C480088401C7B491F
:106F300008807B48008803F04BFB7A49C888FEF73D
:106F400096FB05467849FEF7B7F90446774801688D
:106F50002046FEF758F97549086075480078002802
:106F600060D102217348FFF781FF002850D1012230
:106F7000D10305200007FFF786FF6A49C888FEF79E
:106F800076FB05466849FEF797F904466A480168AA
:106F90002046FEF738F96849086068496648006885
:106FA000FEF732FC3ED2FA2401252BE00A212046CE
:106FB000FEF7B4F8002905D10121C9030520000717
:106FC000FEF7D4FF02215B48FFF750FF002800D0F6
:106FD0000025002D13D102215648FFF747FF002856
:106FE0000DD105F0E9FA01214E484030818005F0CD
:106FF0005BFB642004F0D8FC51485249C8600A2069
:1070000004F0D2FC2046611ECCB20028CED109E0AB
:1070100000220121C90305200007FFF734FF0020EB
:1070200045490860002148480068FEF7EDFB15D28D
:1070300046480088FEF71BFB054629467F20C00511
:10704000FEF73AF90446404801682046FEF730F959
:107050003D49086002203E49087002E000203C499A
:10706000087002213348FFF701FF002819D12D498C
:10707000C888FEF7FCFA05462B49FEF71DF90446C1
:107080002D4801682046FEF7BEF82B4908603149BB
:1070900029480068FEF7B8FB06D829482949C86086
:1070A00002E00020244908602B4920480068FEF7D0
:1070B000ABFB03D201202949087002E000202749D8
:1070C00008701849498F481EFEF7C6FA044617484B
:1070D00001682046FEF78EFB07D82148007800287B
:1070E00003D001201F49087002E000201D490870EC
:1070F0000C49488FFEF7BBFA04460C48016820464D
:10710000FEF778FB05D216480078002801D005F07C
:1071100017FA70BDA6010020650100207E01002045
:1071200004010020EC0D002000007A44A80100209A
:107130009401002000040050A00100200000404005
:107140000400FA0500ED00E0AC010020740100200D
:10715000400100200000A0400000F0423601002065
:107160007A01002045010020704710B50446002C2C
:1071700001D1012010BD02212E200155204601F031
:10718000FBFD204600F0F4F800212E20015500BF41
:107190002D20015500BF0020ECE77047704710B567
:1071A000044620680068C007C00F012148404840DD
:1071B00000280CD0206880680840484048400028DB
:1071C00005D00120216848602046FFF7A3FE206813
:1071D000006802210840400800280BD02068806821
:1071E00008404008002805D0022021684860204659
:1071F000FFF78EFE20680068042108408008002800
:107200000BD02068806808408008002805D0042042
:1072100021684860204600F00DF9206800680821C8
:107220000840C00800280BD0206880680840C008CB
:10723000002805D00820216848602046FFF794FF09
:107240002068006810210840000900280BD0206841
:10725000806808400009002805D010202168486097
:107260002046FFF756FE20680068202108404009AC
:1072700000280BD02068806808404009002805D00D
:107280002020216848602046FFF788FF20680068BA
:1072900040210840800900280BD020688068084001
:1072A0008009002805D04020216848602046FFF76B
:1072B00074FF10BD70B50446002C01D1012070BDD3
:1072C0006068012800D100BF26496069884200D06B
:1072D00000BF2E20005D002805D100212D20015582
:1072E000204600F059F802212E2001552068C5687B
:1072F0006068012803D08905A06A884203D11E2155
:1073000028468843054617496069884201D01648D7
:10731000054016480540A16860680843216A084393
:10732000616A0843A16A084305436068012804D0E4
:107330000121C905A06A884203D1E1682069084398
:10734000054308496069884205D06169A06908431E
:10735000E169084305432068C56001212E200155DD
:107360000020ACE7FFFF00003F1FFFFFF8F119FF0F
:1073700010B5044606492068884208D10548806B4C
:1073800040004008034988630D2000F065F810BDF7
:10739000007C00400010024010B5044609492068F6
:1073A00088420DD10848806B490508430649886327
:1073B000002201210D2000F067F80D2000F058F8A0
:1073C00010BD0000007C004000100240014608682B
:1073D000C069704710B5034602242E20C4541448D7
:1073E000006824072043124C20601868C0680124FC
:1073F000E40420431C68E06018688068012420438E
:107400001C68A06018680069012420431C68206182
:107410001868816118684261186800690424204373
:107420001C68206101242E20C454002010BD0000DF
:1074300000040140704700000648406B01210843EA
:10744000044948630846806B09040843014988637E
:10745000704700000010024000BFC206D20E01219A
:107460009140024A116000BF7047000080E100E0D7
:1074700000BFC206D20E01219140024A116000BF36
:107480007047000000E100E070B504460D46164666
:107490002946204601F0DEFE70BD00000249496821
:1074A0008143014A51607047007000400348006802
:1074B000FF21013108430149086070470070004016
:1074C000024949680143014A516070470070004019
:1074D000074800680221084305490860054800691B
:1074E000042108430349086100BF00BF30BF704753
:1074F0000070004000ED00E010B5024600200E4B89
:107500001868800880000346134318460A4B186029
:107510000A4B1B6904242343084C2361012901D130
:1075200030BF02E040BF20BF20BF044B1B690424D2
:10753000A343024C236110BD0070004000ED00E049
:10754000F8B5044620212068084020287CD1206816
:107550000840202800D100BF00278148806B01210E
:1075600009070840002805D17D48806B08437C4905
:10757000886301277B480068FF210131084000280B
:1075800016D178480068084376490860FFF782FC06
:10759000064606E0FFF77EFC801B642801D9032025
:1075A000F8BD70480068FF21013108400028F1D083
:1075B0006B480568032109050D4060680840A84232
:1075C0000DD0091160680840884208D164480068FD
:1075D000012149040840884201D10120E0E76048C8
:1075E000403000690321090408400546002D3DD0C4
:1075F00060680840A84239D020212068084020282F
:1076000034D15748403000690321090488430546B6
:107610005348403000690121C904084350494031B2
:107620000861084600690121C90488434C4940317A
:10763000086108460561801528408915884215D1E2
:10764000FFF728FC064608E039E0FFF723FC801B23
:107650004549884201D90320A2E7414840300069EA
:10766000012149020840400A0028EED000BF00BFB7
:10767000032109046068084088420AD1384800683C
:107680000901884303221205616811400843344907
:10769000086000BF3248403000690322120461686C
:1076A000114008432E494031086100BF012F05D128
:1076B0002B48806B890588432949886300BF20785F
:1076C000C007C00F002809D025484030C068800896
:1076D0008000A168084322494031C8600221206827
:1076E0000840022809D11E484030C0680C21884358
:1076F000E16808431A494031C86004212068084005
:1077000004280AD116484030C06803218902884302
:107710002169084312494031C860082120680840A7
:1077200008280AD10E484030C06803210903884365
:10773000616908430A494031C860802120680840D7
:1077400080280AD106484030C06803218904884354
:10775000A169084302494031C860002020E70000C9
:10776000001002400070004088130000F8B5044685
:107770000D46002C01D10120F8BD79480068C007F2
:10778000C00FA8420ED27648006840084000284347
:107790007349086008460068C007C00FA84201D0BE
:1077A0000120E9E7022120680840022807D16D483E
:1077B000C068F0218843A16808436A49C8602078FE
:1077C000C007C00F00284CD06068022809D1654866
:1077D0000068012149040840400C002824D1012000
:1077E000CAE76068032809D15E480068012149069C
:1077F0000840400E002817D10120BDE7606801282D
:1078000008D15848006804210840800800280BD19E
:107810000120B1E753480068012149020840400AAD
:10782000002801D10120A7E74E48C06880088000E9
:10783000616808434B49C860FFF72CFB0646606847
:1078400002280FD107E0FFF725FB801B464988423D
:1078500001D9032090E74348C0680C21084008285C
:10786000F1D134E0606803280FD107E0FFF712FB85
:10787000801B3D49884201D903207DE73948C06813
:107880000C2108400C28F1D121E0606801280FD1BB
:1078900007E0FFF7FFFA801B3349884201D9032034
:1078A0006AE73048C0680C2108400428F1D10EE096
:1078B00007E0FFF7EFFA801B2B49884201D903202C
:1078C0005AE72848C0680C2108400028F1D1244814
:1078D0000068C007C00FA8420ED9214800684008C0
:1078E000400028431E49086008460068C007C00FD2
:1078F000A84201D001203FE7042120680840042865
:1079000008D11848C068072109028843E168084384
:107910001449C860082120680840082809D1114886
:10792000C0680721C90288432169C90008430D497D
:10793000C86000F049F80B49C968F02211400909F4
:107940000A4A515CC8400A4908600020FFF7C6FA9D
:107950000746002F01D038460EE700200CE7000054
:10796000002002400010024088130000CAC700082F
:10797000B80100200148006870470000B8010020ED
:1079800000B5FFF7F7FF0549C96807221202114049
:10799000090A034A515CC84000BD000000100240C3
:1079A000DAC7000800B5FFF7E5FF0549C9680722F7
:1079B000D2021140C90A034A515CC84000BD000010
:1079C00000100240DAC70008FEB52E48C7680C2038
:1079D0003840002845D0042804D008280CD00C28B2
:1079E0003ED10BE02748006810210840002801D054
:1079F000254C00E0254C41E0254C3FE00F20800461
:107A00003840800C23490E5C032080053840800DEF
:107A1000401C01901B48C06801210904084000284F
:107A200007D01B49714308460199FDF761FB0546E4
:107A300014E01448006810210840002807D01249BB
:107A4000714308460199FDF753FB054606E00F49CF
:107A5000714308460199FDF74BFB05462C460DE0A6
:107A600000BF08484068072149030840400B0090C8
:107A70000098401C01218140CC0300BF00BF20467C
:107A8000FEBD00000010024000093D000024F4008B
:107A900000127A00E2C70008FEB50446002C01D1AE
:107AA0000120FEBDF848C6680C210E40C7680121C0
:107AB00009040F402078C007C00F002872D0082E9C
:107AC00004D00C2E0FD1084687420CD1EE48006836
:107AD000012149040840400C002863D06068002858
:107AE00060D10120DDE700BF012109046068884200
:107AF00005D1E54800680843E349086027E005210F
:107B00000904606888420ED1DF48006801218904B9
:107B10000843DD490860084600680121090408435C
:107B2000D949086013E0D848006801210904884356
:107B3000D549086008460068012109040840009002
:107B400000BFD148006889008843CF49086000BF62
:107B50006068002813D0FFF79DF9054606E0FFF79F
:107B600099F9401B642801D903209AE7C6480068A8
:107B7000012149040840400C0028F0D012E0FFF732
:107B800089F9054606E0FFF785F9401B642801D90D
:107B9000032086E7BC480068012149040840400CE6
:107BA0000028F0D102212068084002287AD1E0683C
:107BB0000290042E03D00C2E34D1002F32D1B248C3
:107BC0000068042108408008002804D0029800289A
:107BD00001D1012065E7AC4840681F2109028843B4
:107BE000216909020843A84948600846006809213C
:107BF000884302990843A4490860FFF7E5FEA249BB
:107C0000C968F02211400909A04A515CC840A04946
:107C100008600020FFF762F901900198002841D028
:107C200001983EE70298002824D09748006809216F
:107C300088430299084394490860FFF72BF90546E9
:107C400006E0FFF727F9401B022801D9032028E7A7
:107C50008D4800680421084080080028F1D08A4837
:107C600040681F21090288432169090208438649A7
:107C7000486017E084480068400840008249086076
:107C8000FFF708F9054606E0FFF704F9401B022854
:107C900001D9032005E77C480068042108408008DA
:107CA0000028F1D1102120680840102867D1002E4B
:107CB00036D17548006849010840400A002804D0C0
:107CC000A069002801D10120EBE66F484068072138
:107CD00049038843216A08436B4948600846406865
:107CE0000002000A217F0906084367494860206AAC
:107CF000400B401C01218140C8036349C968F02240
:107D000011400909614A515CC8406149086000207E
:107D1000FFF7E4F80190019800284BD00198C0E6E5
:107D2000A06900282CD058480068FF210131084381
:107D300055490860FFF7AEF8054606E0FFF7AAF8D8
:107D4000401B022801D90320ABE64F4800680121FF
:107D500049020840400A0028F0D04B4840680721FB
:107D600049038843216A08434749486008464068F8
:107D70000002000A217F090608434349486019E0D0
:107D800041480068FF21013188433F490860FFF7FF
:107D900081F8054606E0FFF77DF8401B022801D96F
:107DA00003207EE638480068012149020840400A65
:107DB0000028F0D1082120680840082839D16069DE
:107DC00000281BD0304840300069012108432E496B
:107DD00040310861FFF75EF8054606E0FFF75AF804
:107DE000401B022801D903205BE627484030006988
:107DF0000221084040080028F0D01AE02248403014
:107E0000006940084000204940310861FFF742F80E
:107E1000054606E0FFF73EF8401B022801D9032083
:107E20003FE6194840300069022108404008002818
:107E3000F0D1042120680840042879D10020009066
:107E40001148806B89060840002806D10E48806BD7
:107E500008430D498863012000900E480068FF2107
:107E60000131084000281ED10A480068084309492A
:107E70000860FFF70FF805460EE0FFF70BF8401B10
:107E8000642809D903200CE600100240CAC7000884
:107E9000B80100200070004085480068FF210131D2
:107EA00008400028E9D000BFFF210131A0688842C6
:107EB00005D18048006908437E49086130E0A06828
:107EC00000280DD17B480069FF21013188437949A1
:107ED00008610846006909158843764908611FE072
:107EE00005210902A06888420DD17248006901216C
:107EF000890208436F4908610846006989150843EB
:107F00006C4908610CE06B480069FF21013188432E
:107F10006849086108460069091588436549086190
:107F200000BFA068002815D0FEF7B4FF054608E0A2
:107F300031E0FEF7AFFF401B5F49884201D90320C3
:107F4000AFE55C480069012149020840400A002869
:107F5000EFD013E0FEF79EFF054607E0FEF79AFF1D
:107F6000401B5549884201D903209AE551480069D0
:107F7000012149020840400A0028EFD10098012859
:107F800008D14C484038806B012109078843494992
:107F90004039886300BF606A00284CD00C2E69D03D
:107FA000606A022848D14348403800680121090628
:107FB0008843404940390860FEF76CFF054606E0FB
:107FC000FEF768FF401B022801D9032069E5394804
:107FD00040380068012149060840400E0028EFD1D2
:107FE000E16AA06A0843216B084332494039C968F5
:107FF000FD221204914308432E494039C8600846C7
:1080000000680121090608432A4940390860FEF743
:1080100041FF054606E0FEF73DFF401B022801D95F
:1080200003203EE523484038006801214906084006
:10803000400E0028EFD038E01E484038006801218B
:10804000090688431B4940390860FEF723FF0546AF
:1080500006E0FEF71FFF401B022801D9032020E5A0
:10806000144840380068012149060840400E0028A5
:10807000EFD11AE0606A012800D112E50D484038BE
:10808000C768012000043840A16A88420BD10F2044
:1080900080043840E16A884205D1032080053840D9
:1080A000216B884201D00120FBE40020F9E40000AC
:1080B00000700040401002408813000010B50446D4
:1080C000002C01D1012010BD606A002800D100BF42
:1080D0000021A1625120005D002804D150200155EB
:1080E000204600F035F80221512001552068006833
:1080F0004021884321680860A16860680843E168FE
:108100000843216908436169084301225202A169B9
:1081100011400843E1690843216A0843A16A084302
:1081200021680860A069000C04210840616A0843C6
:10813000216848602068C069910088432168C8614F
:10814000002060650121512001550020BBE700009F
:1081500010B586B00446142101A8FDF73CF8144977
:108160002068884222D11348406B89140843114982
:10817000486300BF0846C06A012108430D49C86230
:108180000846C06AC007C00F009000BF00BFE020D3
:108190000190022002900020039003200490002010
:1081A000059001A905200007FEF76AFD06B010BD85
:1081B000003001400010024070B504462546681E9C
:1081C0000949884201D901200CE0681E074948612D
:1081D0000321081F01F03EF80020044988610720B0
:1081E0000861002070BD0000FFFFFF0000E000E01C
:1081F00070477047FEB504462068C5692068066868
:10820000206887682807000F0190019800280ED188
:108210002020284000280AD020203040002806D006
:10822000206E002802D02046216E8847FEBD0198AE
:1082300000287DD0F807C00F002804D1FF2021308E
:1082400030400028F5D0E807C00F00280BD0FF20F1
:1082500001303040002806D0012021680862E06F1C
:1082600001210843E0670220284000280AD0F807CF
:10827000C00F002806D0022021680862E06F0421A8
:108280000843E0670420284000280AD0F807C00F00
:10829000002806D0042021680862E06F022108430C
:1082A000E0670820284000280ED020203040002819
:1082B00003D1F807C00F002806D008202168086203
:1082C000E06F08210843E067E06F002846D02020D7
:1082D0002840002809D020203040002805D0206EFA
:1082E000002802D02046216E8847E06F0090206869
:1082F000806840210840402804D0082100980840A8
:10830000002826D0204602F0E2FC20688068402148
:108310000840402819D12068806888432168886017
:10832000E06E00280DD02548E16E8863E06E00E025
:1083300015E0FEF77BFA002810D0E06E816B8847CD
:108340000CE02046FFF755FF08E02046FFF751FFFD
:1083500004E02046FFF74DFF0020E06766E70120BC
:108360000005284000280CD0012080053840002856
:1083700007D001200005216808622046FFF738FF7A
:1083800054E78020284000280AD080203040002870
:1083900006D0606E002802D02046616E884745E70F
:1083A00040202840002807D040203040002803D03B
:1083B000204602F09EFC39E700BF37E70DAC00080D
:1083C00010B50446002C01D1012010BDA069002881
:1083D00000D000E000BF606F002805D100217020B0
:1083E0000155204600F02CF82420606720680068C2
:1083F0004008400021680860204602F04DFD012839
:1084000000D1E2E7606A002802D0204602F070FA4C
:10841000206840680921C9028843216848602068B3
:1084200080682A21884321688860206800680121CB
:10843000084321680860204602F0D2FAC5E7000030
:1084400010B586B00446142101A8FCF7C4FE3649D5
:108450002068884266D13548406B01218903084372
:108460003249486300BF0846C06A012108432F49CA
:10847000C8620846C06AC007C00F009000BF00BFB6
:10848000032040020190022002900020039003206C
:1084900004900420059001A905200007FEF7F0FBD9
:1084A0002348244908600320486000212148816056
:1084B000C160802101610021416181612021C16190
:1084C00009020162FEF764FA002801D0FDF7FCFB07
:1084D00000BF1848E066846200BF1548143816498A
:1084E0000860032048601021134881600021C160AA
:1084F00080210161002141618161C1610162FEF75A
:1085000047FA002801D0FDF7DFFB00BF0A48A0664C
:10851000846200BF002201211B20FEF7B5FF1B2053
:10852000FEF7A6FF06B010BD003801400010024063
:1085300030000240F41700203C18002070B50446BB
:108540000D461646A06F202863D1002D01D0002EC5
:1085500001D1012070BD01210903A068884208D122
:108560002069002805D1E807C00F002801D00120AC
:10857000F0E700BF7020005D012801D10220E9E78B
:1085800001217020015500BF656558200653002069
:10859000E0672220A067E06E002820D01E48E16E30
:1085A000C8621E48E16E08631D48E16E4863002002
:1085B000E16E88632368194624313346626DE06EAC
:1085C000FEF73AFA00280AD01020E06700BF002129
:1085D0007020015500BF202060670120BAE700BF6E
:1085E00000217020015500BF20680068FF21013183
:1085F00008432168086020688068012108432168D9
:1086000088602068806840210843216888600020D5
:10861000A0E702209EE7000077AC0008C1AC00088C
:1086200025AC000810B50346986F20287DD100299D
:1086300001D0002A01D1012010BD01242403986833
:10864000A04208D11869002805D1C807C00F00282A
:1086500001D00120F0E700BF7020C05C012801D1EB
:108660000220E9E701247020C45400BF5965582056
:10867000C2525A20C2520020186600BF24039868D4
:10868000A0420AD11869002803D1294C5C20C452A9
:1086900024E0FF245C20C45220E0986800280AD11E
:1086A0001869002803D1FF245C20C45216E07F24FF
:1086B0005C20C45212E0012424079868A0420AD129
:1086C0001869002803D17F245C20C45206E03F24AF
:1086D0005C20C45202E000245C20C45200BF002091
:1086E000D8672220986718688068012420431C6896
:1086F000A060012424039868A04205D118690028CD
:1087000002D10C48186601E00B48186600BF00242F
:108710007020C45400BF18680068FF24213420432F
:108720001C682060002087E7FFE7022084E7000044
:10873000FF010000C1AD00082DAE00087047704772
:10874000FFB583B004460D461746606F202875D1EB
:10875000002D01D0002F02D1012007B0F0BD012172
:108760000903A068884208D12069002805D1E807DC
:10877000C00F002801D00120EFE700BF7020005D8E
:10878000012801D10220E8E701217020015500BF36
:108790000020E06721206067FEF77CFB01905020FD
:1087A00007535220075301210903A068884205D1CD
:1087B0002069002802D10026029502E02E46002002
:1087C000029021E006980090002280212046019B23
:1087D00002F050FD002801D00320BEE7002E09D191
:1087E00002980088C005C00D216888620298801C2C
:1087F000029003E0307821688862761C5220005B8A
:10880000401E81B2522001535220005B0028D9D172
:1088100006980090002240212046019B02F02AFD8C
:10882000002801D0032098E72020606700BF0021C6
:108830007020015500BF00208FE7FFE702208CE782
:108840007047000002E002480249C860FBE70000F0
:108850000400FA0500ED00E010B500220421052017
:108860000007FEF710FB0022082105200007FEF795
:108870000AFB0A2003F0A2F80122042105200007C8
:10888000FEF701FB0A2003F099F8002204210520DD
:108890000007FEF7F8FA10BD10B5002204210520EC
:1088A0000007FEF7F0FA0122082105200007FEF775
:1088B000EAFA0A2003F082F80122042105200007C9
:1088C000FEF7E1FA0A2003F079F8002204210520DE
:1088D0000007FEF7D8FA10BD70B505460024002643
:1088E0001EE00022042105200007FEF7CCFA0A2032
:1088F00003F064F80122042105200007FEF7C3FA03
:108900006006040E082105200007FEF7AFFA0028D4
:1089100001D0601CC4B2052003F050F8701CC6B230
:10892000082EDEDB002D02D1FFF7B6FF01E0FFF7D6
:1089300093FF204670BD70B5044600220421052037
:108940000007FEF7A0FA00252AE080202040C01191
:10895000002806D00122082105200007FEF793FA1F
:1089600005E00022082105200007FEF78CFA6006CA
:10897000040E0A2003F022F801220421052000073A
:10898000FEF781FA0A2003F019F8002204210520DD
:108990000007FEF778FA0A2003F010F8681CC5B249
:1089A000082DD2DB70BD10B501220821052000077B
:1089B000FEF769FA0122042105200007FEF763FA99
:1089C0000022082105200007FEF75DFA0A2002F0C8
:1089D000F5FF0022042105200007FEF754FA10BD20
:1089E00010B50022042105200007FEF74CFA0022F2
:1089F000082105200007FEF746FA0A2002F0DEFFF4
:108A00000122042105200007FEF73DFA012208217A
:108A100005200007FEF737FA0A2002F0CFFF10BD4D
:108A200010B500240122082105200007FEF72BFACB
:108A3000062002F0C3FF0122042105200007FEF7F3
:108A400022FA062002F0BAFF07E0601CC4B2FA2C3A
:108A500003DDFFF7C5FF012010BD08210520000739
:108A6000FEF704FA0028F0D10022042105200007B7
:108A7000FEF709FA0020EFE738B501F0E9FF02F050
:108A80003BF868480068C069FDF778FA0446664814
:108A9000808F00282DD065480078002806D0012856
:108AA0000AD0022817D0032822D11BE0012291020C
:108AB0005F48FEF7E8F91BE0212C06DA00220121CD
:108AC00089025B48FEF7DFF904E001229102584871
:108AD000FEF7D9F90CE00022012189025448FEF783
:108AE000D2F905E0012291025148FEF7CCF900BF0E
:108AF00000BF0121C9024E48FEF7B8F9002828D06E
:108B000000204C4908604C480078002804D101201E
:108B10004949087002F0F6FB4848007863280BDDED
:108B2000002208214248FEF7AEF90122D1030520B8
:108B30000007FEF7A8F91BE0012208213C48FEF7D8
:108B4000A2F900220121C90305200007FEF79BF9C5
:108B50000EE0002038490870002208213448FEF752
:108B600092F900220121C90305200007FEF78BF9C5
:108B70002D484030808C012821D1002530480090BC
:108B800072B680212F48FDF7BBF80546002D05D0B1
:108B9000022269462B48FDF7A5F9054662B62AA0D0
:108BA00002F0BAFC002120484030818403F07CFDB3
:108BB000642002F0F9FE28482849C86000BF1A481E
:108BC0004030408C01280ED10021174840304184AC
:108BD00000201549088003F067FD642002F0E4FEE0
:108BE0001D481E49C86010484030008C01280BD138
:108BF00000210D484030018403F056FD642002F04E
:108C0000D3FE15481549C8600748008814498842B2
:108C100003D10548C088002802D10F480F49C86019
:108C200038BD000074170020EC0D0020400100202A
:108C300000040050A80100207C01002064010020F5
:108C4000AAAA0000384A0008BDF8C8EBC9FDBCB6A6
:108C5000C4A3CABD0D0A00000400FA0500ED00E03F
:108C6000AA55000008B53721202000F073F8032131
:108C7000212000F06FF84021222000F06BF808213D
:108C8000232000F067F8AA21302000F063F80A489A
:108C9000008FC1B2322000F05DF80221332000F0D5
:108CA00059F85F21202000F055F8684600F006F8DA
:108CB0000A2002F083FE08BDEC0D002010B504462A
:108CC00021460F2000F023F8002800D110BD01201C
:108CD000FCE770B504460025FFF765FE3220FFF77C
:108CE0002AFEFFF79DFEE0B2FFF725FEFFF798FE94
:108CF000FFF759FE3320FFF71EFEFFF791FE00201D
:108D0000FFF7EAFD0546FFF76BFE284670BD70B51C
:108D100005460C462846FFF7DCFF2070012070BD99
:108D200070B504460D46FFF73EFE3220FFF703FE06
:108D3000FFF776FEE0B2FFF7FEFDFFF771FE284673
:108D4000FFF7F9FDFFF76CFEFFF74AFE0A2002F07D
:108D500035FE70BD70B504460D4629462046FFF726
:108D6000DFFF012070BD000010B50248FEF717FAC2
:108D700010BD0000EC160020F0B585B004460020C0
:108D8000039072B64F4920684018002806D14E481B
:108D9000C068032189040840039000E000BF00BFC1
:108DA0002068806802902068C0680190206845694A
:108DB0002068866943492068401800280DD1424840
:108DC0004038806A490508433F494039886208466F
:108DD000806A40004008886200E000BF00BF002DAC
:108DE00001D1002E5FD0374920684018002807D1F4
:108DF0003548C0680321890488433349C86000E0CE
:108E000000BF00BF002D1DD020680069012108436C
:108E10002168086120684561FEF73CF8074600BFFD
:108E2000FEF738F8C01B0090206800680821084051
:108E3000082804D07D21C90000988842F0D9082074
:108E400021684860002E1DD0206800690121084378
:108E50002168086120688661FEF71CF8074600BF9C
:108E6000FEF718F8C01B0090206800681021084029
:108E7000102804D07D21C90000988842F0D9102024
:108E8000216848600F4920684018002809D10E4821
:108E9000C068032189048843039908430A49C860CC
:108EA00000E000BF00BF2068006940084000216862
:108EB000086102982168886001982168C86062B6DC
:108EC00005B0F0BD0084FFBF401002401CB500207B
:108ED000009001901E481F49086000211D48C16391
:108EE000012080071B49486000211A488160072142
:108EF0008163012101610021C160001D017741777B
:108F0000001F8162FF21C2314162002124300172C1
:108F10000421243841610021016381614163C16101
:108F2000FDF784FA002801D0FCF7CEFE0A48009035
:108F30008013019069460748FDF7ECF9002801D03D
:108F4000FCF7C2FE00210348FDF776F91CBD0000C6
:108F500000240140901600200200000408B500BF64
:108F60000A48006B01210843084908630846006B62
:108F7000C007C00F009000BF00BF002201210A20DF
:108F8000FEF782FA0A20FEF773FA08BD00100240CD
:108F900000B587B0142102A8FCF71DF900BF654891
:108FA000C06A042108436349C8620846C06A0421B4
:108FB0000840019000BF00BF00BF5E48C06A80212A
:108FC00008435C49C8620846C06A80210840019095
:108FD00000BF00BF00BF5748C06A01210843554980
:108FE000C8620846C06AC007C00F019000BF00BF3A
:108FF00000BF0846C06A022108434E49C8620846BD
:10900000C06A02210840019000BF00BF01221C215C
:1090100005200007FDF737FF012247494748FDF7C4
:1090200032FF002246494548FDF72DFF00229121DD
:10903000090205200007FDF726FF012002904148A4
:1090400003900020049002A905200007FDF718FEF8
:1090500002200290032003900020049002A9052022
:109060000007FDF70DFE0C20029011200390002058
:1090700004900320059002A905200007FDF700FEDB
:1090800010200290012003900020049002200590FF
:1090900002A905200007FDF7F3FD01200290112031
:1090A000039000200490059002A92448FDF7E8FDF4
:1090B00002200290244803900120049002A91F4836
:1090C000FDF7DEFD2148029001200390002004906E
:1090D000059002A91948FDF7D3FD0120C0020290B6
:1090E000002003900220049002A91448FDF7C8FD57
:1090F000912000020290012003900020049005902E
:1091000002A905200007FDF7BBFD8020029000208A
:1091100003900120049002A90848FDF7B1FD002248
:1091200001210520FEF7B0F90520FEF7A1F907B0EF
:1091300000BD0000001002400106000000040050C5
:109140000830000000001110000021100836000057
:1091500010B50A480A490860002048600021084804
:109160008160084941610021016241628162FEF72C
:10917000A1F8002801D0FCF7A7FD10BD007C00403D
:10918000EC160020FFFF000010B5124812490860DD
:10919000FF200530486000210F488160C1600161F7
:1091A00041610121490281610021C1610162416285
:1091B00081620721C162FEF781FF002801D0FCF720
:1091C00083FD05480068006840210843024909689A
:1091D000086010BD003001401C17002000B585B0AC
:1091E00014216846FBF7F7FF164817490860E1208D
:1091F00040024860002114488160C16001610C2177
:10920000416100218161C161016230200E494862E3
:10921000012109030C4881634900C163FFF7D0F8BD
:10922000002801D0FCF750FD012208490648FFF74D
:10923000F9F9002801D0FCF747FD02F05DF805B010
:1092400000BD0000003801407417002062010020BA
:109250007047000010B5002819DA1A4A03071B0FDF
:10926000083B9B089B00D2588307DC0EFF23A340DA
:109270009A438B071B0E8407E40EA3401A43114B3D
:109280000407240F083CA408A4001A5118E00E4A51
:1092900003231B02D21883089B00D2588307DC0EDD
:1092A000FF23A3409A438B071B0E8407E40EA340C1
:1092B0001A43054B032424021B198408A4001A51E5
:1092C00010BD00001CED00E000E100E000BF00BFA9
:1092D00000BFBFF34F8F00BF00BF00BF0648074964
:1092E000C86000BF00BF00BFBFF34F8F00BF00BF0B
:1092F00000BF00BF00BFFDE70400FA0500ED00E07D
:10930000F0B58FB000200E900A2002F0D5FE7D202F
:10931000C00002F0EDFE0020FE490870FE48007813
:109320000C2802DB0B20FC490870012251020520A9
:109330000007FDF7A8FD0020F8490870F8480078FC
:10934000F8490871F84800784000F849097808435E
:10935000F749097889000843F249C871F54801784E
:109360000068401CF34A1060C8B2EE49C870F24869
:1093700000788874F04800784200F049E9481330DA
:10938000FBF710FF0620E7494872ED480078887225
:10939000EC48007808730846EB490A78427049782F
:1093A0008170E54909784900084615300022DD49F9
:1093B00002F0A0FFE0490978490008461530002175
:1093C00002F0ACFF022002F0D1FE0020D549C871A6
:1093D000DE490870DE4908700120DE49087000206F
:1093E000DD490870DD48FDF7F1FFDD490880002008
:1093F000CA490870D0480078FCF739F90646FCF7EE
:10940000B5F9D84AD84B05910490FCF745F8079177
:10941000069002F065FA002201239B07099108904B
:10942000FBF788FF0B910A90FCF782F9C0B20D9010
:109430000D984001CA4909884018CC49088008465F
:1094400000880121C903884204DBC8480088401A0B
:10945000C6490880C648C7490860C7480078401C0C
:10946000C5490870BD48FDF7B1FFC449088063E2F3
:10947000BA48FDF7ABFFC149088013E0B748FDF7D4
:10948000A5FFBE49088008460088B8490988884277
:1094900008DBBA480088B5490988B94A8918884262
:1094A00000DA09E000210F2002F064FDB5490860F0
:1094B000B54908400028E1D000BFB2480068401C10
:1094C000002801D1FFF702FFAE480068012189039F
:1094D000084000287DD08122D20100210F2002F017
:1094E000C2FE7D20C00002F003FE002002F0AFFDAE
:1094F0000021102002F03EFD4006400EA349086006
:109500000846008881B20022A14802F083FDA048ED
:10951000407A0728ABD102229E499D48401DFBF7A7
:1095200065FE0028A3D102F056FF9B4A03C202F059
:109530003BFF9A4A03C279480078401C774908707B
:109540009348427808A90A74817808A8417468464B
:10955000008E7D49098888427ED191498C48C08916
:10956000088090488A49098A01807C48FDF72EFFCF
:109570008249088002F0D4FB8848036840688A4A20
:1095800000219A1848410106170A0F43790849003B
:1095900000200A0E000210430B02002211469A1806
:1095A000484182490A6048607B480CC85D480A30DF
:1095B00002F0E0FE6049097889001631594A88189E
:1095C00076490CC902F0D6FE78480CC855481230CE
:1095D00000E0A2E102F0CEFE08205249487256494E
:1095E0000978890008461C3000224E4902F082FEAC
:1095F00051490978890008461C30002102F08EFE8E
:10960000384602F051FD012002F0B0FD68490870B3
:1096100002216848FDF72AFC002801D1012000E062
:109620000020424908706449594842890A8080896B
:109630004880084600684F4908605548C07C0007CC
:10964000000F032805D05248C07C0007000F5B497B
:1096500008704F48C07C00E026E1001158490870AE
:10966000002045490870012039490870414948489F
:1096700042890A808089488051480078002818D0A3
:10968000022244494248401DFBF7B0FD002810D19A
:1096900001202E4908702349C8713C4800781638CB
:1096A0004849087008460278394916314648FBF7A0
:1096B00079FD0120284908703A480088FF30C330FE
:1096C00038490880084600884049884212DD3548FC
:1096D0000088401A3349088031480088401C3049CE
:1096E0000880084600887D21C900884202DB0020EE
:1096F0002B4908802A4800887D21C9004843294910
:1097000009884018324908603248007832490870A8
:10971000324965E0F10000203201002011010020F3
:10972000640100206012002036010020B0010020FA
:109730004501002074000020300100205A14002050
:1097400074010020040100200A01002034010020DF
:10975000240100202601002025010020EC16002015
:109760002A010020B81E85EB51B8CE3F2C01002005
:10977000A08601000C01002021010020280100200A
:10978000983A00007800002000D0272448010020EB
:10979000B012002058010020800000208800002026
:1097A00060010020FC000020000062029000002008
:1097B000F0000020000400500001002040010020C3
:1097C000410100203501002058150020E70300006A
:1097D000140100207E0100203301002082010020BE
:1097E0000988302251430846FBF736FFC0490990EB
:1097F00009880A2251430846FBF72EFF0890099971
:10980000FBF75AFD7F21C9050A90FBF7FCFC0B9082
:10981000FBF756FFB7490880B7480078401E098813
:10982000884202D10120B5490870B1480088B44986
:109830000880B4490020085EFBF720FF09910890DA
:10984000B1480088FBF72EFFB04AB14B0191009060
:10985000FBF722FE05910490AE480068FBF70EFF6F
:1098600003910290059B049AFBF708FE079106906E
:10987000099B089AFBF75EFD0B910A90FBF734FFFA
:10988000A5490860A548008800F0A2FEA448007819
:10989000002808D100BF00210F2002F06BFB8021BF
:1098A00008400028F7D056E06846008EFCF748FBD9
:1098B000064603209B4988559B499C4842890A805B
:1098C00080894880B0009A4940189849898A018067
:1098D00095480068B100974A5050B1001631964A39
:1098E000881896490CC902F045FDB0009049085807
:1098F0008D49096888420FDDB0008D49085800285D
:109900000AD089480068002806DD6846008E8C4928
:10991000088002208B4908700EE08B4A00210F203E
:1099200002F0A1FC8948017889480078401C8142F6
:1099300002D0002002F08BFB73480088854909881B
:10994000884200DA94E57048008882490988824A92
:1099500089188842F6DC00BF02F0E2F97A4A002159
:109960000F2002F080FC00246E480078002803D10C
:109970006A48008800F02CFE002078490870002515
:1099800023E06848405D00281DDD74480078401CD5
:10999000724908706348405DA100714A50506800E8
:1099A0007049085A6100704A5052A80061490A582B
:1099B0002146601CC4B288006C490A505948405D79
:1099C000401E58494855681CC5B261480078854218
:1099D000D7DB5E480078032803DA604800785F49E7
:1099E00008705E4800786249087000253FE0002456
:1099F00036E0A0005D490958601C80005B4A1058A1
:109A000081422BDDA200594B99586200564B985A5F
:109A1000AA00534B9A580C92621C9200534B9A58CE
:109A2000A300524EF250621C52004F4B9A5A6300F0
:109A30004D4EF252621C9200494B9A58A300484E78
:109A4000F250621C9200494B9950621C5200464BE6
:109A50009852631C9B000C9AF25000BF601CC4B269
:109A600043480078401EA042C3DC681CC5B2404891
:109A70000078401EA842BADC3E4800880A214843CC
:109A80003D490978884202DA00202E4908703B4897
:109A9000007800281CD000200C9000260B9038483D
:109AA00000780B903648467880780C900B98022806
:109AB0000DD1344988193249C91C0C9AFBF772FB45
:109AC00002F0F2FD642001F06FFFFFF7FFFB00BF23
:109AD0001D4A803200210F2002F0C5FB0022012127
:109AE000490205200007FDF7CEF90FB0F0BD0000D8
:109AF000600100207E0100203301002025010020AC
:109B00002E0100203C01002028010020F853E3A58D
:109B10009B843E40140100201C0100200401002011
:109B2000F00000204C15002000010020B0120020A1
:109B30008C140020BC14002060120020880000203B
:109B40000A0100206800002000D027241101002015
:109B5000300100202C010020983A00003201002042
:109B60001C1500205A14002072140020EC14002050
:109B70003101002074010020210100203401002067
:109B800058150020EC0D002070470000F0B58FB094
:109B9000DA4F0020C0430E9000200C900A2002F003
:109BA0008BFA7D20C00002F0A3FA0020D44908708F
:109BB000002681E1D348867300220146142002F07A
:109BC00099FB0021142002F0A9FB022002F0CEFA3A
:109BD00000BF00210F2002F0CDF9CB490860CB492E
:109BE00008400028F5D0C8480068401C002801D172
:109BF000FFF76CFBC4480068012189030840002876
:109C00007ED08122D20100210F2002F02CFB002106
:109C1000102002F0AFF945066D0E29460022BC481F
:109C200002F0F8F9BA48407A02286AD10222B9490A
:109C3000B748401DFBF7DAFA0028F6D102F0CBFB5B
:109C4000B54A03C202F0B0FBB44A03C20C98002824
:109C50002CD101200C90B249AD48C0890880B14890
:109C6000AB49098A0180B048FDF7B0FBAF490880D5
:109C7000AC480088FF30C330AA49088008460088F5
:109C8000AB49884212DDA7480088401AA5490880E0
:109C9000A3480088401CA249088008460088A449BF
:109CA0000B31884202DB00209D4908809848428998
:109CB00069468A868089C88604229549491C9D4840
:109CC000FBF770FA954803684068FF2252040021B0
:109CD0009A1848410106140A0C43204602F0E4F9A0
:109CE0006108490000200A0E000210430B02002206
:109CF00011469A18484190490A604860864801E038
:109D0000D0E0CBE00CC88B48093002F033FB83482D
:109D10000CC888480D3002F02DFB87480CC88548D8
:109D2000113002F027FB00228249491E3C2002F03C
:109D3000E1FA00213C2002F0F1FA012002F016FACB
:109D40007E4908706E480078401C6D4908700121FA
:109D5000C90305200007FCF709F9714800887D2137
:109D6000C90048436F49098840187549086075481B
:109D70000078754908706A4800880A3800B273494B
:109D8000088008460021415E002906DA00887D210E
:109D9000C900401800B26D4908806D490988302219
:109DA00051430846FBF758FC684909900020085EBB
:109DB000FBF752FC08900999FBF77EFA7F21C90551
:109DC0000A90FBF720FA0B90FBF77AFC5D490880BC
:109DD0005D480078401E0988884202D101205D4913
:109DE00008704F4800885C4908805C490020085E84
:109DF000FBF744FC099108904C480088FBF752FCA3
:109E0000574A584B01910090FBF746FB059104908F
:109E10004B480068FBF732FC03910290059B049AC3
:109E2000FBF72CFB07910690099B089AFBF782FA37
:109E30000B910A90FBF758FC4B4908604B4800888F
:109E400000F0C6FB0D98B84212DA0D9800280FD02A
:109E500004222F49491C0EA8FBF7A4F9022044490B
:109E60000870444800780A214843434908700D9F10
:109E700032480078002808D100BF00210F2002F0EE
:109E800079F8802108400028F7D0802200210F2097
:109E900002F0E9F90020394908700BE00120374948
:109EA000087007E0364A00210F2002F0DCF901209B
:109EB00032490870701CC6B2032E00DA7AE60C989C
:109EC000002815D129480088002805D02748008897
:109ED0002C490988884203DD2A48008823490880E4
:109EE00022480088401E284909884843274908809D
:109EF00027490E9808800FB0F0BD00003F420F00C8
:109F0000F1000020EC1100207800002000D0272470
:109F1000B01200205801002080000020880000209E
:109F200060010020FC000020EC1600202801002029
:109F3000E70300000F12002090000020F000002036
:109F4000140100207E010020330100203E0100208A
:109F500082010020250100202E0100203C0100206C
:109F6000F853E3A59B843E401C010020040100201F
:109F7000680000207401002010010020C4000020AF
:109F8000009027246C0100206A0100206601002057
:109F90000A010020F8B555485549086002F00CFB4D
:109FA0002120000153494880112088800846403014
:109FB00000795149087008460078002809D17D20B1
:109FC000C0004C49C8800120C8870A20488700206B
:109FD00088874848C088002802D164204549C88045
:109FE0004448008F0A2802DD022042490887414880
:109FF000C08E3C2802DD3C203E49C8863D48C08ECC
:10A00000002802DA00203B49C8863A48C08E3B4906
:10A0100008703848C08F3A4908703648808F3949EF
:10A0200008703448807A3849087032488088374947
:10A0300008600520364908802E49C88834490988B7
:10A04000FBF76CF8334908802A4988883149098828
:10A05000FBF764F82E480088414388B22E490880F7
:10A0600009887D22D20051430846FBF707FB0446CE
:10A070002A4A2B4BFBF778FA0646FBF759FB29498E
:10A08000088025480088284908801A48C1887D2012
:10A09000C000FBF743F82549088008460188C8201E
:10A0A000FBF73CF822490880012022490880FBF791
:10A0B00065FF214908801B4802880121C9031F4808
:10A0C000FDF788F9002801D0FBF7FEFD0F48016875
:10A0D0001BA001F021FA0748C1881DA001F01CFA5D
:10A0E000044801891FA001F017FAF8BD41B3000828
:10A0F00050000020EC0D0020940100200100002001
:10A100007A0100207B01002063010020580100201B
:10A110006A0100206C01002066010020F853E3A5CD
:10A120009B843E40720100207601002074010020D3
:10A13000820100207E01002078010020EC16002022
:10A14000B1EAC7A949443A202564202E0D0A00002F
:10A15000CDA8D1B6BCE4B8F43A202564206D732EA6
:10A160000D0A0000B5A5B4CECDA8D1B6BBF9D5BEB9
:10A17000CAFDC1BF3A202564B8F62E0D0A000000C2
:10A18000F0B589B00120B849088008460188C82088
:10A19000FAF7C4FFB5490880B5480078401CB449B7
:10A1A00008700878C10F091849104900411A0AD0EF
:10A1B000B04801880088401EAE4A1080022902DAA9
:10A1C000C82011460880AB48008800F001FA0A2038
:10A1D00001F072FF7D20C00001F08AFF0221A64835
:10A1E000FCF744FE002801D1012000E0002080009F
:10A1F000A249097849000843A14909780843A149BF
:10A20000887210204872A048C1887D20C000FAF7EB
:10A2100085FF9C4948739D480078887308469A4991
:10A220008A78C272C9780173974920310A7EC27355
:10A23000497E0174944922310A7E4274497E8174B8
:10A2400000220146152002F055F80021152002F0E9
:10A2500065F8022001F08AFF01E0FEF70DFC002105
:10A260000F2001F087FE8A4908608A4908400028CB
:10A27000F3D087480068401C002801D1FFF726F87A
:10A280008348006801218903084000287ED081228C
:10A29000D20100210F2001F0E6FF0021102001F083
:10A2A00069FE4006400E7C4908600846008881B27D
:10A2B00000227A4801F0AEFE7848407A112865D134
:10A2C000022277497548401DFAF790FF0028F6D121
:10A2D0007248427808A90A70807848706F48807A7E
:10A2E0006149088008460188C820FAF717FF5F49CE
:10A2F00008806A48007B5F4908806A496748C089CE
:10A30000088069486549098A01806848FDF75EF858
:10A310006749088064480088FF30C330624908807C
:10A32000084600886349884212DD5F480088401A69
:10A330005D4908805B480088401C5A4908800846EF
:10A3400000885C490B31884202DB002055490880B7
:10A35000544800887D21C900484353490988401862
:10A360005549086055480078554908704D4800889F
:10A370000A3800B25349088008460021415E00298E
:10A3800008DA00887D21C900401800E069E000B2C9
:10A390004C49088035490988302251430846FBF76B
:10A3A0005BF9064647490020085EFBF755F907466A
:10A3B0003146FAF781FF05467F21C905FAF723FFE9
:10A3C0000446FBF77DF93D4908803D480078401E72
:10A3D0000988884202D101203B4908703148008831
:10A3E0003A4908803A490020085EFBF747F9059191
:10A3F00004902F480088FBF755F90646354A364B3E
:10A40000FBF74AF8019100902B480068FBF736F9FA
:10A410000446019B009AFBF731F803910290059BDB
:10A42000049AFAF787FF07910690FBF75DF92B492D
:10A4300008606846008C2A4908801848807C2949B1
:10A440000870084600784200144913312648FAF78C
:10A45000A9FE08480088FF2802D00320234908707D
:10A4600000BF09B0F0BD000074010020820100208F
:10A470005001002004010020000400507A01002057
:10A480007B01002060120020EC0D00200100002064
:10A490007800002000D0272448010020B0120020BE
:10A4A0005801002060010020FC000020EC16002074
:10A4B00028010020E7030000140100207E01002095
:10A4C000330100203E010020250100202E01002044
:10A4D0003C010020F853E3A59B843E401C01002072
:10A4E0000A010020300100205A14002068000020DA
:10A4F00000B585B014216846FAF76DFE00220121EF
:10A50000C9031048FCF7BFFC0120C00300900120E4
:10A51000019000200290039069460A48FCF7B0FBC6
:10A520000120C003009003200190002002900390BE
:10A5300069460448FCF7A4FB022001F035FA05B097
:10A5400000BD0000000400507047000038B504460C
:10A550000D460020009055201B490870AA20487025
:10A5600003208870601DC87003200871084645717B
:10A5700084716800154A811822461348C01DFAF7F5
:10A5800011FE002008E0811C0F4A525C69460988D0
:10A5900051188AB20092401C611D8842F3DB0A48C0
:10A5A000801CFBF7B5FA0090E01D0749411868468A
:10A5B00000780870684640784870214609310248A2
:10A5C00000F0B0FB38BD00002C160020EC0D002080
:10A5D0007CB5064606E02F4800882F490988401AB6
:10A5E0002C4908802B4800882B4909888842F2DAD8
:10A5F0002848008829490988484380192849088043
:10A6000024480088132807D1224800882349098854
:10A610004843801922490880214800883021484356
:10A620006430642148431F490860084600681E4999
:10A630000968401A4B21090140181C490860084666
:10A640000068FBF71BF80446194A1A4BFAF78CFF0F
:10A6500001910090FBF748F8174908600846006828
:10A660000121C903884204DD13480068401A1249D9
:10A67000086011480068002806DA0F4800680121C8
:10A68000C90340180C4908600B4800680B49096869
:10A6900048617CBD7E010020740100208201002001
:10A6A00080010020900100201C0100208C0100206E
:10A6B000F853E3A59B843E4088010020EC1600205F
:10A6C00001460020054A126890B2054A1040024631
:10A6D0000A431046014A10607047000000300140F4
:10A6E000C7FF000010B5FCF7DBFB10BD00B599B04B
:10A6F00034210CA8FAF76FFD142107A8FAF76BFDB7
:10A700001C216846FAF767FD244800680321C90246
:10A7100088430121C902401820490860FCF7C6FEA1
:10A720001F4800690321C90288431D4908610620AA
:10A730000C9088150E9001200F9010201090022090
:10A7400015900021169141041791410518910CA80C
:10A75000FDF7A2F9002801D0FBF7B6FA0F20079009
:10A7600003200890002009900A900B90012107A86F
:10A77000FCF7FCFF002801D0FBF7A6FA812000902F
:10A78000002002900320800406906846FCF7D8FE63
:10A79000002801D0FBF798FA19B000BD0070004006
:10A7A0004010024015480068FF2101310843134959
:10A7B00008600846C068124908401049C860084649
:10A7C0000068104908400D49086008468068400844
:10A7D00040008860084600680121890488430749D1
:10A7E00008600846C068FD21090488430349C86021
:10A7F0000020086104480549886070470010024045
:10A800000C40FF88F6FFF6FE0050000800ED00E067
:10A8100010B51020052109078862AF20800001F0E3
:10A82000CDF8102005210907886101F0BDFB2C49F6
:10A83000086003E001F0B8FB294908602848006877
:10A8400028498842F6D128480078002806D00128F7
:10A8500014D0022822D003283ED13AE00122D103AD
:10A8600005200007FCF70FFBFFF78AFC00220121FF
:10A87000C90305200007FCF706FB2DE00122D103E8
:10A8800005200007FCF7FFFAFFF780F900220121FD
:10A89000C90305200007FCF7F6FA1DE0134800780D
:10A8A000401E124908700122D10305200007FCF761
:10A8B000EAFAFBF785FB00220121C9030520000706
:10A8C000FCF7E1FA09480078002801D10649087030
:10A8D00002E0FEF715FD00BF00BF01F005FA10BD54
:10A8E0004C0100203001CADE680000201001002069
:10A8F000818CC907C90F002908D001684968012265
:10A9000052049143826A1143026851600222416AF3
:10A910001140022907D101684968D2039143C26AF4
:10A920001143026851600422416A1140042907D191
:10A930000168496812049143026B11430268516037
:10A940000822416A1140082907D1016849681203A9
:10A950009143426B1143026851601022416A1140D9
:10A96000102907D10168896812029143826B114353
:10A97000026891602022416A1140202907D10168B4
:10A98000896812029143C26B1143026891604022B0
:10A99000416A1140402915D10168496892039143E9
:10A9A000026C11430268516001221205016C914250
:10A9B00008D101684968032252059143426C114352
:10A9C000026851608022416A1140802907D10168E4
:10A9D000496812039143826C1143026851607047C9
:10A9E00038B504460020E067FCF754FA05462068B5
:10A9F00000680821084008280BD114482B46002283
:10AA000089040090204600F035FC002801D0032086
:10AA100038BD206800680421084004280BD10B4889
:10AA20002B46002209050090204600F023FC002858
:10AA300001D00320ECE720206067A06700BF002161
:10AA40007020015500BF0020E2E70000FFFFFF017A
:10AA500070B50025C82420480078002800D070BDBB
:10AA60001E480078002800D0F9E701201B49087033
:10AA70001B48406B002801D10870F0E71848406B74
:10AA8000C8210D1A1CE01749174A1268885C17493B
:10AA900009688847164800880A21484315490880F4
:10AAA00011480068401C1049086008460068C82822
:10AAB00001DB002008600A48406BC8210D1A641EA3
:10AAC00009480068A84201D0002CDCDC00200349C2
:10AAD000087000BFC3E700004A0000204C000020BF
:10AAE00000000240240D0020400000205000002003
:10AAF000740100209C01002010B53A48007800281D
:10AB000003D139480078002800D010BD0120364913
:10AB100008703648C06980210840002802D13249B7
:10AB20000870F2E7324900200856324900228A565E
:10AB3000904215D12D48C0694021084000280BD013
:10AB40002D480078002807D000202B4908702B489A
:10AB50000088401C29490880002023490870D4E758
:10AB600025480078002805D10120234908700A20D3
:10AB700000F024FF1F4900200856CC2148432049FB
:10AB80004018001D1F490968405C184988621D482B
:10AB90000068401C1B490860164900200856CC215B
:10ABA00048431749085817490968884214DC0020AF
:10ABB000144908600F480078401C40B20D490870E5
:10ABC000084600780E2801D1002008700E48007851
:10ABD000401C40B20C49087000200349087000BFB7
:10ABE00093E700004A0000204B000020003801409D
:10ABF0003D0000203C0000204D0000205A000020B5
:10AC0000FC010020600000203E00002070B50546D9
:10AC1000AC6A00215A200153522001532046FDF70F
:10AC2000E8FA70BDF8B50546AC6A666FA76F206894
:10AC3000806880210840802807D1212E05D100217D
:10AC400052200153204600F064F8206880684021BB
:10AC50000840402807D1222F05D100215A20015356
:10AC6000204600F034F8E06F10210843E0672046EA
:10AC7000FDF7BFFAF8BD70B50546AC6A28680068F4
:10AC800020210840002817D100215A2001532068B4
:10AC90000068FF21013188432168086020688068CE
:10ACA000400840002168886020688068402188430F
:10ACB000216888602020A0672046FDF73FFD70BD19
:10ACC00070B50446A56A2846FDF739FD70BD0168D8
:10ACD0000968FF2221329143026811600168896886
:10ACE00049084900026891602021816700210166BE
:10ACF000704710B5044620680068402188432168E9
:10AD0000086020206067002060662046FDF798FDFF
:10AD100010BD01680968C0229143026811602021BA
:10AD20004167704770B505460C46204800780028FA
:10AD300003D11F480078002800D070BD01201B49B6
:10AD40000870C82C04DC1B4800214156002903DC94
:10AD5000002016490870F0E7174900200856CC215A
:10AD6000484316490C50144A00215156CC225143F5
:10AD7000124A8918081D22462946FAF713FA0E4886
:10AD80000078401C40B20C490870084600780E2834
:10AD900001D10020087007480078401E40B20549E4
:10ADA000087000200149087000BFC6E74A00002073
:10ADB0004B0000203E0000203D000020FC01002050
:10ADC000F8B504465C20075BA06F222827D12068D5
:10ADD000406A86B2656D304638402880606D801CC0
:10ADE00060655A20005B401E81B25A200153005B0F
:10ADF00000281AD120680068FF212131884321688A
:10AE00000860206880684008400021688860202031
:10AE1000A067002020662046FDF790FC05E0206832
:10AE200080690821084321688861F8BD70B504462F
:10AE30005C20065BA06F222827D12068406A85B27B
:10AE4000F0B22840616D0870606D401C60655A204A
:10AE5000005B401E81B25A200153005B00281AD1CA
:10AE600020680068FF21213188432168086020683C
:10AE7000806840084000216888602020A06700208A
:10AE800020662046FDF75AFC05E02068806908210D
:10AE900008432168886170BDF0B587B00446102072
:10AEA00004900025002003900026E749206888428E
:10AEB00000D100E000BF2169A06808436169084330
:10AEC000E1690843074620680068E04908403843C4
:10AED0002168086020684068032109038843E1680D
:10AEE000084321684860A769D7492068884201D093
:10AEF000206A0743206880680B2109028843384391
:10AF00002168886000BFD249206888421CD1D1489E
:10AF1000C0688007800F002806D001280AD00228C8
:10AF200005D003280CD108E0012004900BE002209A
:10AF3000049008E00420049005E00820049002E05A
:10AF40001020049000BF46E0C349206888421CD10D
:10AF5000C048C0680C210840002806D004280AD048
:10AF6000082805D00C280CD108E0002004900BE044
:10AF70000220049008E00420049005E008200490DA
:10AF800002E01020049000BF25E0AF49206888420D
:10AF90001FD1B048C068032189020840002808D0AA
:10AFA00001218902401A0AD0401A05D0401A0CD15A
:10AFB00008E0002004900BE00220049008E0042048
:10AFC000049005E00820049002E01020049000BFE7
:10AFD00001E01020049000BF9B492068884256D1B0
:10AFE000049804281AD004DC002807D002281CD1B9
:10AFF00008E0082816D0102817D117E0FCF7C0FC8D
:10B00000064616E0934840380068102108400009C1
:10B01000002801D0914E00E0914E0AE0FCF7D4FCEC
:10B02000064606E00126F60303E000BF0120039078
:10B0300000BF00BF002E0AD0606841004018B04237
:10B0400003D860680003B04202D201200390F4E00C
:10B05000606802903046FF21013100F084FA626896
:10B06000520800238018594101910090029AFAF782
:10B0700069F8054603200002854205D379488542D8
:10B0800002D82068C560D8E001200390D5E00121F6
:10B09000C903E06988426FD1049804283CD006DCDB
:10B0A000002809D0012813D002284AD11CE0082822
:10B0B0003ED0102845D145E0FCF762FC40006168B5
:10B0C0004908401802906168FAF712F885B23CE02E
:10B0D000FCF768FC4000616849084018029061680C
:10B0E000FAF706F885B230E05A4840380068102177
:10B0F00008400009002807D061684A085A4BD01858
:10B10000F9F7F6FF85B206E061684A08574BD01898
:10B11000F9F7EEFF85B218E0FCF756FC40006168D5
:10B120004908401802906168F9F7E2FF85B20CE027
:10B1300061684A0801231B04D018F9F7D9FF85B2CA
:10B1400003E000BF0120039000BF00BF102D0FD30C
:10B15000474885420CD846480F38284005902807B4
:10B16000400F05990843059005982168C86064E080
:10B170000120039061E0FFE7049804283AD006DC40
:10B18000002809D0012812D0022847D11AE0082847
:10B190003BD0102842D142E0FCF7F2FB616849083D
:10B1A000401802906168F9F7A3FF85B23AE0FCF716
:10B1B000F9FB61684908401802906168F9F798FF47
:10B1C00085B22FE02348403800681021084000096C
:10B1D000002807D061684A08204BD018F9F788FF8B
:10B1E00085B206E061684A081D4BD018F9F780FF68
:10B1F00085B217E0FCF7E8FB616849084018029047
:10B200006168F9F775FF85B20CE061684A080123AF
:10B21000DB03D018F9F76CFF85B203E000BF012013
:10B22000039000BF00BF102D05D31148854202D8FE
:10B230002068C56001E00120039000202066606660
:10B24000039807B0F0BD000000480040F369FFEF2D
:10B2500000380140401002400044004000093D0019
:10B260000024F400FFFF0F0000127A000048E801FC
:10B27000FFFF0000FFB581B004460D4617460A9E49
:10B2800022E0701C00281FD0FBF704FE0499401A2E
:10B29000B04201D8002E17D120680068FF21A131EB
:10B2A0008843216808602068806840084000216861
:10B2B000886020206067A06700BF002170200155D2
:10B2C00000BF032005B0F0BD2068C0692840A84237
:10B2D00001D1012000E00020B842D2D00020F1E7E7
:10B2E00010B510200349096808620248FCF782FF84
:10B2F00010BD0000741700200D2001490870704730
:10B300003E00002010B50A4800880A214843094938
:10B310000880FDF723FEFDF761FFC82206490748B4
:10B32000FDF70CF9002801D0FAF7CEFC10BD0000A3
:10B33000740100209C010020240D002074170020BF
:10B3400070B50446002569480078082864D100BF1C
:10B35000002004E06649095C49198DB2401C65492A
:10B360000978491F8142F5DC63480078281885B2C6
:10B3700060480078281885B260480078281885B29F
:10B380005F480078281885B25E480078281885B292
:10B390006019C0B2FF2835D157480078012827D05E
:10B3A00002282DD15849554A1278881854490A78EC
:10B3B0004F49F9F7F7FE01F077F9642000F0F4FA4D
:10B3C00000BF00BF00BF00BF00BFBFF34F8F00BF73
:10B3D00000BF00BF4D484E49C86000BF00BF00BF5E
:10B3E000BFF34F8F00BF00BF00BF00BF00BFFDE72E
:10B3F00042480078411042480078FFF7A7F800E083
:10B4000000BF00BF0020394908703C490870394925
:10B4100008704049087068E034480078072812D165
:10B4200033483C49097844543A480078401C39492B
:10B43000087030480078401F0978884255D10820AC
:10B440002A49087051E029480078062805D12C487F
:10B45000047007202549087047E024480078052833
:10B4600005D1264804700620204908703DE01F4899
:10B470000078042805D12048047005201B49087075
:10B4800033E01A480078032808D11A4804700020D5
:10B490001A49087004201549087026E013480078FE
:10B4A000002805D1552C03D10120104908701CE05B
:10B4B0000E480078012805D1AA2C03D102200B499F
:10B4C000087012E009480078022807D1032C05D142
:10B4D0000320064908700B48047006E00020034969
:10B4E0000870064908700349087070BD51010020BA
:10B4F000C8150020530100205601002054010020EF
:10B500005201002055010020EC0D00200400FA0536
:10B5100000ED00E0570100200FB410B503A9044B63
:10B52000044A029800F034F910BC08BC04B0184773
:10B5300091C30008BC0100202021020C01D0102181
:10B540001046020A01D010460839020901D01046FF
:10B55000091F820801D01046891E420801D0881EAA
:10B560007047081A7047F8B582B28BB2040C0D0C04
:10B5700010465843002126465E43370C3604801996
:10B58000794116466E43370C3604801979412646B8
:10B590006E438919F8BD30B47446641E2578641C66
:10B5A000AB4204D3635D5B00E31830BC18471D4613
:10B5B000F8E702E008C8121F08C1002AFAD1704754
:10B5C0007047002001E001C1121F002AFBD1704723
:10B5D00008B5002100916B46012202212C2000F0C9
:10B5E00057FE022100916B4601222C2000F050FEF4
:10B5F00008BD000038B504466D2000906B4601225E
:10B6000008492E2000F044FE002C05D0064A0749C8
:10B610002E2000F017FE04E0054A04492E2000F019
:10B6200011FE38BD060800000706000006180000DD
:10B630000716000038B504466B460222002136206A
:10B6400000F0B8FC2300FFF7A6FF0E11081A5454AF
:10B650005454233154543D444B54002168460170E6
:10B660004078FE2108406946487043E06946087802
:10B67000FC21084001210843694608703AE0694608
:10B680000878FC210840022108436946087031E02F
:10B6900068460078B321084048210143684601709C
:10B6A0004078802108436946487023E06846017865
:10B6B000B32001406846017040784106490E684653
:10B6C000417017E06946487802210843694648708E
:10B6D00010E069464878FD2108406946487009E055
:10B6E00069460878CF210840202108436946087040
:10B6F00000E000BF00BF6B4601220021362000F0B1
:10B70000C7FD00AB013301221146362000F0C0FD19
:10B7100038BD08B5032168464170012101706B46B0
:10B7200002220021362000F0B3FD0122D2030621BF
:10B730002D2000F087FD012000F036F90120FFF7F1
:10B7400079FF08BD38B504462004010E68464170F3
:10B7500004706B46022204212D2000F099FD032184
:10B76000684601706B46012206212D2000F090FDF5
:10B770000021684601706B46012206212D2000F051
:10B7800087FD0A212D2000F0F5FB0546284638BD2F
:10B79000FFB58DB00446002506E025280AD0109A92
:10B7A0000F999047641C6D1C20780028F5D128461D
:10B7B00011B0F0BD00270121484A009700E007437F
:10B7C000641C23780846203B98401042F7D120782B
:10B7D0002E2817D1042007436078641C2A280CD136
:10B7E0000E98641C02C800910E900BE000990A228A
:10B7F000514330394018641C00902078014630399C
:10B800000929F3D920780028D1D0642808D06928E4
:10B8100006D075281ED0109A0F9990476D1C5BE0DA
:10B820000A200E99019001C90E91002802DA4042C7
:10B830002D2102E0390504D52B216A461172012120
:10B8400003E0F90704D02021F7E70BAE0B910DE0E0
:10B850000021FAE70A200E99019001C90E91F7E73D
:10B860000199F9F745FC3031761E31700028F7D187
:10B8700003A8801B20300190780701D5009801E0D3
:10B88000012000900199884201DD401A00E000206B
:10B890000027009006E002A8109AC05D0F9990471B
:10B8A0006D1C7F1C0B988742F5DB04E0109A30205A
:10B8B0000F9990476D1C0099481E00900029F5DCF7
:10B8C00005E03078109A761C0F9990476D1C01990D
:10B8D000481E01900029F4DC641C65E7092801007A
:10B8E000F8B54A002B4B520DD6182B4A0C4605468C
:10B8F000142E2BDA002E12DA284BF9F71BFD00224A
:10B900001346F9F747FF40D2002C03DA0124E4077D
:10B9100000253AE02046284337D0214C14E0214F3F
:10B920000B46F7403B402B4331D01C4BF9F702FD4F
:10B9300000221346F9F72EFF27D2002C03DD012049
:10B940000005F0400419BC4300251EE0332E1EDC28
:10B9500033460027143BFF43DF40384217D00F4BDC
:10B96000F9F792FD00221346F9F714FF0DD2002CCF
:10B970000ADD142E0CD03420811B01208840401990
:10B98000A84200D2641C0546BD4321462846F8BDA6
:10B99000641CF9E701FCFFFF9C7500883CE4377EDE
:10B9A0000000F03FFFFF0F0070B504467D20C0008F
:10B9B00060430546284600F001F870BD002100BF35
:10B9C00040E000BF00BF00BF00BF00BF00BF00BF1E
:10B9D00000BF00BF00BF00BF00BF00BF00BF00BF6F
:10B9E00000BF00BF00BF00BF00BF00BF00BF00BF5F
:10B9F00000BF00BF00BF00BF00BF00BF00BF00BF4F
:10BA000000BF00BF00BF00BF00BF00BF00BF00BF3E
:10BA100000BF00BF00BF00BF00BF00BF00BF00BF2E
:10BA200000BF00BF00BF00BF00BF00BF00BF00BF1E
:10BA300000BF00BF00BF00BF00BF00BF00BF00BF0E
:10BA400000BF491C8142BCD370470000F0B585B0EF
:10BA500004460020049003902578607940008A49CC
:10BA6000085A02906078401E8849C6B20863042DC7
:10BA700001D0072D01D1012000E0002001902078A5
:10BA800082490873E07900280AD1084680690121BB
:10BA9000890508437D4988610298C010029006E03C
:10BAA0007A48806901218905884378498861207A2C
:10BAB0007649487308468069217A090403221204F2
:10BAC00011400843714988610846002182690420B9
:10BAD00000F0C9FB6E492E20029A00F0B3FB3046FD
:10BAE000FFF788FD6B48405D810040186A494318A4
:10BAF000052207212B2000F0CBFB684901980B1889
:10BB000001220B21282000F0C3FB6248405D800029
:10BB100063490A580C21282000F0A5FBE079800039
:10BB200060494018A1794900425A0221272000F0BB
:10BB300089FB70005C490A5A0421272000F082FB2F
:10BB4000E079002805D164220621272000F07AFB45
:10BB50001EE0A07804280DD11020009010220621AC
:10BB6000272000F06FFB6B4601222621272000F0E2
:10BB70008FFB0DE02820009020220621272000F0D6
:10BB800061FB6B4601222621272000F081FB00BFCC
:10BB9000300146494018E1788900425808212720A1
:10BBA00000F061FBA17A627A08021043002803D1F9
:10BBB0003F496172090AA172A17A637A08021843A7
:10BBC00002462021272000F03DFB3A480C21026864
:10BBD000232000F048FB71003648001D425A042122
:10BBE000232000F02FFBA07900280BD0E079324908
:10BBF000431801220021212000F04AFB0320049079
:10BC0000012003902807000F2901F022114008436A
:10BC100061788904032292041140084304990905BC
:10BC20009200114008430399490401225204114033
:10BC30000843217989051F22920511400843617943
:10BC4000C906C90EC906084307463A4600211F2007
:10BC500000F009FBA0786178084300040B490861F3
:10BC600008460069E17949030122D20311430843E0
:10BC700006490861084600210269082000F0F3FA2D
:10BC8000002005B0F0BD000098C70008C0010020EA
:10BC90000428000040C700080C0000202A000020F3
:10BCA00048C7000868C7000874C7000878C70008BC
:10BCB0004110000060C700082C00002038B5044681
:10BCC0000D460848808B0443224600212C2000F0BA
:10BCD000B9FA00956B46012206212C2000F0D8FA13
:10BCE00038BD0000C001002010B5FFF771FC10BD89
:10BCF00070B505460421362000F03CF90446002DBD
:10BD000003D00120C002044304E00121C9022046FF
:10BD10008843044622460421362000F0A4FA70BD70
:10BD200038B54020009000210E2000F023F9044691
:10BD3000002211460E2000F096FA6B4601220021E7
:10BD40000D2000F0A5FA084A00210F2000F08BFA20
:10BD500000F05CFA224600210E2000F084FA002157
:10BD60000248017338BD0000F8FF2724E0010020DD
:10BD7000FEB50546042001900026002700206B49EF
:10BD80004875086300216948203041710173002023
:10BD9000664988834863886300F006F96349086050
:10BDA00003E000F001F961490860604800686049FB
:10BDB0008842F6D10020FFF73DFC00F0F5F85B4922
:10BDC00008605C480078242805DD5A48007824384B
:10BDD000594908600EE0062156480078F9F79EF9A7
:10BDE0000621081A440153480078F9F797F90C43E3
:10BDF000514804605048007800064F4909880904FA
:10BE000008434D490968090208434B49096808433A
:10BE10004A4908600846002102681E2000F023FA03
:10BE200000F0C2F84149086001AB01220021242042
:10BE300000F02EFA1E20FFF785FC86B230123B4937
:10BE400088730420FFF77EFC074600F0ADF8374901
:10BE50000860F8B200280FD0022000906B46012243
:10BE600012212D2000F014FA3048808B01210903A3
:10BE700008432E49888300BF00F096F82B490860DC
:10BE80000620FFF75FFC294948600720FFF75AFCAE
:10BE900026498860F006C00E08750846007D002817
:10BEA00001D1102008752149087D00F049FAE80702
:10BEB000C00F002809D0FFF72CFC1C48808B012103
:10BEC000C9020843194988830CE00521362000F097
:10BED00039F804461A48044022460521362000F06D
:10BEE000B1F900BF0120FFF7A5FB0021042000F0FD
:10BEF00041F80E4988610021262000F03BF80446F5
:10BF000005208003044380000443224600212620AC
:10BF100000F0A9F900222621362000F093F900F064
:10BF200043F8024908600020FEBD0000C001002067
:10BF30003001CADE010000200400002008000020BB
:10BF4000FFFD0000F8B504460D46094FA9B2A0B2A6
:10BF50006B46022200F02EF80646002E06D16846F7
:10BF60004078010268460078081887B23846F8BD64
:10BF7000FFFF0000FEB505460E460027FF43B1B2A5
:10BF8000A8B201AB042200F015F800900098002838
:10BF900008D1032404E0380201A9095D4718641E92
:10BFA000002CF8DA3846FEBD10B500210846FFF730
:10BFB000E1FF10BDFFB581B006460C4617460025CF
:10BFC000002C04D129466D1C684646541AE04020D6
:10BFD0003043C2B229466D1C684642547F2C04DCB3
:10BFE00028466D1C69460C540CE0E0B280210843E1
:10BFF00029466D1C6A4650546004020E28466D1C8A
:10C0000069460A54A8B23A466946049B00F018FBF8
:10C0100005B0F0BD70B504460D46164623462A46C7
:10C0200031461120FFF7C6FF70BD10B50446234608
:10C03000052200211520FFF7BDFF10BD10B50446F5
:10C040002346052200211720FFF7B4FF10BD38B5A5
:10C0500004460020009000F0D9F8FF250135002C9F
:10C0600001D0680005432A4600210D2000F0EAF8BF
:10C07000002C17D06B46012203210F20FFF79AFFF7
:10C08000684600780821084000280BD0FFF748FEDA
:10C09000FF2501352A4600210D2000F0D3F80020AD
:10C0A000C04338BD0020FCE710B5044622460121FC
:10C0B0000A2000F0D8F810BD70B5054600211A20FE
:10C0C000FFF758FF0446240D24052803000B044302
:10C0D000224600211A2000F0C6F870BD10B50446B3
:10C0E000224602492E2000F0ADF810BD04180000D1
:10C0F00038B504466B46012203210420FFF75AFF9E
:10C10000002C16DD224600210C2000F09BF8694629
:10C1100008781021084300900F48806909060843F9
:10C120000D4988616B4601220321042000F0B0F81C
:10C1300010E069460878102188430090064880691D
:10C1400009068843044988616B46012203210420C3
:10C1500000F09EF838BD0000C001002010B5044674
:10C1600022460021182000F06DF810BDF8B50446F5
:10C1700000250020009000260220204000280AD040
:10C18000802000906B46012200210D2000F080F8F5
:10C1900001211D480173E007C00F002826D0694621
:10C1A00008780621084300906B46012200210D20EB
:10C1B00000F06EF803210F20FFF7C4FE0646812031
:10C1C000C0003040002801D100251AE04020009036
:10C1D0006B46012200210D2000F05AF80020FFF7E5
:10C1E00087FD0021084801734D1E0AE06946087862
:10C1F0000221084300906B46012200210D2000F02F
:10C2000047F82846F8BD0000E00100201CB501AB4E
:10C21000012203210F20FFF7CDFE69460879802116
:10C22000084069460979402211404900884208D0F7
:10C23000012000906B46012203210D2000F028F818
:10C2400000BF1CBDF8B505460E461446684604708E
:10C2500021124170B1B2A8B26B46022200F018F868
:10C2600007463846F8BDFEB506460F46144600257B
:10C2700003E069464C55240A6D1C042DF9DBB9B264
:10C28000B0B26B46042200F003F801900198FEBDA5
:10C29000FFB581B006460C4617460025002C07D195
:10C2A00080203043C2B229466D1C6846425419E0D2
:10C2B000C0203043C2B228466D1C69460A547F2C08
:10C2C00003DC28466D1C0C540CE0E0B280210843CE
:10C2D00029466D1C6A4650546004020E28466D1CA7
:10C2E00069460A54A8B23A466946049B00F0F6F93A
:10C2F00005B0F0BD70B504460E461546281901215B
:10C300008902884202DD0020C04370BDA21E334670
:10C3100029460920FFF7BCFF0020F6E770B5044668
:10C320000D46064800692043A905084306463246E3
:10C3300000210820FFF797FF002070BDC0010020FA
:10C3400038B504466B4601220E212B20FFF732FE42
:10C3500068460078410949010091E106C90E684626
:10C360000078014300916B4601220E212B20FFF73C
:10C370008FFF38BD70B50146002006E00A541E0646
:10C38000140A34431B0A2246401C0428F6DB70BD05
:10C3900013B50C4601231A4669460248FCF7D0F94A
:10C3A00000981CBD741700207CB500210C460D467A
:10C3B0006846FFF73AFE042608E0220E28021043E2
:10C3C000240205466846805D0443761E002EF4DA9A
:10C3D000204629467CBD7CB500210C460D466846AA
:10C3E000FFF72CFE042608E0220E28021043240248
:10C3F00005466846805D0443761E002EF4DA20462A
:10C4000029467CBDFAF754FDFEF770F9FCF7C0FD34
:10C41000FCF79EFEFCF7A2FDFCF7E0FEFCF7B4FE85
:10C42000FCF754FD0122D10305200007FAF72BFD8C
:10C43000FDF7B0FDFCF716FCF9F7E8FBF9F79CFBFC
:10C440000721FF204130FFF739FC344800880A21DA
:10C450004843334908800122110305200007FAF7F9
:10C4600012FDC8222F493048FCF768F8002801D097
:10C47000F9F72AFC50E02D48007800284AD02C48D3
:10C480000078002846D0FEF731F9002027490870CF
:10C49000F9F732FE27490870084600780F280DDDAD
:10C4A000012211032448FAF7EEFCFEF7B1F900224D
:10C4B000012109032048FAF7E6FC0CE001225103B0
:10C4C0001D48FAF7E0FCFEF7A3F900220121490319
:10C4D0001948FAF7D8FCFCF7CFFA11480088002871
:10C4E00004DD0F480088401E0D490880134800787D
:10C4F000002811D10A48008800280DD10121C90265
:10C500000D48FAF7B3FC002806D101210846FAF7D6
:10C51000F3FF01E0FCF7B0FAADE700007401002082
:10C520009C010020240D00207417002065010020CC
:10C530009401002064010020000400504D00002000
:10C5400000B585B01748FAF710FE14216846F8F7D1
:10C5500042FE154800900320019000200290694699
:10C5600005200007FAF78CFB69461048FAF788FBAC
:10C5700069460F48FAF784FB01210846FAF7BCFF29
:10C58000FF200130FAF78AFF0A48006804210843B7
:10C59000084908608815FAF793FFFAF799FF05B084
:10C5A00000BD0000EC160020FFFF0000000400505A
:10C5B000000800500070004010B5012292021D4991
:10C5C0001D48F9F7B8FB1B4800881C49884230D049
:10C5D0000846184908807D20C00088804010C88027
:10C5E0000A200881002048811E20C0438881012044
:10C5F000C88100200884088248828882C882088313
:10C6000088831E20C886022008877820488701205A
:10C610008887C8870021074840300184418481848D
:10C6200000200449C883002102484030818000F086
:10C630003BF810BDEC0D002000FC0008AA550000DE
:10C6400070B504460D460021102005263607B0625D
:10C6500000BF0DE0685C134EF06000BF11488068B9
:10C66000C007C00F0028F9D00E48C0681870491CD8
:10C67000A142EFDB00210DE000200A4EF06000BF78
:10C6800008488068C007C00F0028F9D00548C06876
:10C690005854491C9142EFD3102005263607B0614B
:10C6A000002070BD0030014010B5002472B6012199
:10C6B00089020848F9F724FB0446002C06D0012221
:10C6C000920205490348F9F70DFC044662B620467C
:10C6D00010BD000000FC0008EC0D002070B5044601
:10C6E0000D460021102005263607B06200BF0CE081
:10C6F000685C124EF06000BF10488068C007C00F31
:10C700000028F9D00D48C068491CA142F0DB002187
:10C710000CE0585C094EF06000BF08488068C00714
:10C72000C00F0028F9D00548C068491C9142F0D3D9
:10C73000102005263607B061002070BD0030014092
:10C740000000010203040005405C0000A05C04003E
:10C75000C06C0800805C0400E03F1E00E07D1E000D
:10C7600007A9022570889B880A00160001000600B0
:10C770000100020087008D002D001A3152001A338B
:10C780009A001A351D011A376B003B31BE003B334E
:10C790005E013B3596023B37000099599959EB51A0
:10C7A0008F421E45142E0080EB51F5283333E13AB9
:10C7B000703DE13AC235852BC2353333C235C235BF
:10C7C000AE47E13A5138A330513800000000000074
:10C7D000000001020304060708090000000001022E
:10C7E0000304030406080C10182030000CC80008CD
:10C7F00000000020C0010000E859000848C80008F7
:10C80000C0010020E01A0000C2B50008C1130704EF
:10C81000380D091E080540082609104008560A135D
:10C820001D043B08BE0576D8BC4010080430C84241
:10C83000011B02025E1409010202C98103185C1285
:08C84000022D01023502522015
:04000005080050C1DE
:00000001FF
